:0200000480007A
:10000000B72F0000938F0F8073900F306F00400365
:100010001300000013000000130000001300000094
:100020001300000013000000130000001300000084
:100030001300000013000000130000001300000074
:100040009702000093824211739052309300000097
:10005000130100009301000013020000930200004E
:100060001303000093030000130400009304000036
:10007000130500009305000013060000930600001E
:100080001307000093070000130800009308000006
:100090001309000093090000130A0000930A0000EE
:1000A000130B0000930B0000130C0000930C0000D6
:1000B000130D0000930D0000130E0000930E0000BE
:1000C000130F0000930F000097110200938181C568
:1000D0001705020013050547979503009385456EA4
:1000E00013060000EF00001A170502001305053B78
:1000F000970502009385C54213060000EF008018A3
:1001000017A503001305056C97B503009385456B90
:1001100037B6ABAB1306B6BAEF00C01617B1030083
:100120001301416AEF8050179392120093D212008C
:100130009382D2FF638A02008322010013014100EF
:100140006F0000177300203083220100130141006B
:10015000730020301301C1FF23205100F32220340B
:10016000E3C402FC8322010013014100130141F8A2
:1001700023221100232421002326310023284100BB
:10018000232A5100232C6100232E71002320810299
:10019000232291022324A1022326B1022328C10293
:1001A000232AD102232CE102232EF1022320010570
:1001B0002322110523242105232631052328410567
:1001C000232A5105232C6105232E71052320810745
:1001D000232291072324A1072326B1072328C1073F
:1001E000232AD107232CE107232EF107732520347E
:1001F000F3251034130601006F000000731015344E
:1002000083204100032181008321C10003220101D9
:1002100083224101032381018323C10103240102BD
:1002200083244102032581028325C10203260103A1
:1002300083264103032781038327C1030328010485
:1002400083284104032981048329C104032A010569
:10025000832A4105032B8105832BC105032C01064D
:10026000832C4106032D8106832DC106032E010731
:10027000832E4107032F8107832FC1071301C10775
:10028000730020302320C5006376B50013054500B8
:100290006FF05FFF678000000000000000000000BA
:1002A000000000000000000000000000000000004E
:1002B000130101F8232011002322210023243100FF
:1002C0002326410023285100232A6100232C71009A
:1002D000232E8100232091022322A1022324B10294
:1002E0002326C1022328D102232AE102232CF10272
:1002F000232E010323201105232221052324310568
:100300002326410523285105232A6105232C710545
:10031000232E8105232091072322A1072324B1073F
:100320002326C1072328D107232AE107232CF1071D
:100330009702020083A2C21923A02200F3221034E4
:10034000232E5106EF00C03B170102000321411884
:10035000032101008322C10773901234B7220000E9
:100360009382028873A00230832001000322C1001F
:100370008322010103234101832381010324C1015D
:100380008324010203254102832581020326C10241
:100390008326010303274103832781030328C10325
:1003A000832801040329410483298104032AC10409
:1003B000832A0105032B4105832B8105032CC105ED
:1003C000832C0106032D4106832D8106032EC106D1
:1003D000832E0107032F4107832F81071301010893
:1003E00073002030970202009382C21523A01200EE
:1003F00023A2220023A4320023A6420023A85200F5
:1004000023AA620023AC720023AE820023A09202D2
:1004100023A2A20223A4B20223A6C20223A8D202CC
:1004200023AAE20223ACF20223AE020323A01205A8
:1004300023A2220523A4320523A6420523A85205A0
:1004400023AA620523AC720523AE820523A092077E
:1004500023A2A20723A4B20723A6C20723A8D20778
:1004600023AAE20723ACF207EF60906117010200B4
:1004700003210106032101008322C1077390123476
:10048000B72200009382028873A00230832001000B
:100490000322C1008322010103234101832381013F
:1004A0000324C10183240102032541028325810223
:1004B0000326C10283260103032741038327810307
:1004C0000328C103832801040329410483298104EB
:1004D000032AC104832A0105032B4105832B8105CF
:1004E000032CC105832C0106032D4106832D8106B3
:1004F000032EC106832E0107032F4107832F810797
:1005000013010108730020309702020093828203D6
:1005100083A0020003A1420083A1820003A2C200C3
:1005200083A2020103A3420183A3820103A4C201A7
:1005300083A4020203A5420283A5820203A6C2028B
:1005400083A6020303A7420383A7820303A8C2036F
:1005500083A8020403A9420483A9820403AAC20453
:1005600083AA020503AB420583AB820503ACC20537
:1005700083AC020603AD420683AD820603AEC2061B
:1005800083AE020703AFC20983AF82076780000012
:1005900073700430130101F823201100232221007D
:1005A000232431002326410023285100232A6100FF
:1005B000232C7100232E8100232091022322A102EB
:1005C0002324B1022326C1022328D102232AE102D7
:1005D000232CF102232E01032320110523222105C0
:1005E000232431052326410523285105232A6105AB
:1005F000232C7105232E8105232091072322A10797
:100600002324B1072326C1072328D107232AE10782
:10061000232CF1079702020083A282EB23A0220081
:10062000232E1106EF30006317010200032141EA77
:10063000032101008322C10773901234B722000006
:100640009382028873A00230832001000322C1003C
:100650008322010103234101832381010324C1017A
:100660008324010203254102832581020326C1025E
:100670008326010303274103832781030328C10342
:10068000832801040329410483298104032AC10426
:10069000832A0105032B4105832B8105032CC1050A
:1006A000832C0106032D4106832D8106032EC106EE
:1006B000832E0107032F4107832F810713010108B0
:1006C00073002030737004306F00000073104530E9
:1006D000678000007325403073F04330678000006E
:1006E00097070000938747FE232EB5FE2322C5FA05
:1006F000232635F82320F5F8130505F86780000058
:10070000130101FF23261100EF605034EF20500B3E
:10071000631805008320C1001301010167800000F8
:100720008320C100130101016F30C052930785007F
:100730001307F0FF2322F5002324E5002326F5000C
:100740002328F500232005006780000023280500EA
:10075000678000008327450023A2F50003A78700D8
:1007600023A4E50003A787002322B70023A4B70032
:1007700023A8A50083270500938717002320F500F1
:100780006780000003A605009307F0FF13078500AC
:100790006316F6006F008003138707008327470066
:1007A00083A60700E37AD6FE23A2F50023A4B700B0
:1007B00023A4E5002322B70023A8A5008327050072
:1007C000938717002320F5006780000003270501A9
:1007D000832747006FF05FFD0327450083268500D0
:1007E000832705012324D70003278500832645009E
:1007F0002322D70003A747006316A700032785001D
:1008000023A2E7002328050003A507001305F5FF31
:1008100023A0A70067800000032605049387050036
:10082000630406028325C50003274500B385C50080
:100830002326B50063E6E500832505002326B500E1
:10084000138507006F50C07C67800000130101FF13
:100850002324810023261100130405002322910084
:10086000EF30907283278404635AF0048327440294
:1008700063860704930444026F0000028327840404
:100880009387F7FF2324F404832784046358F0023A
:10089000832744026384070213850400EF30D01DD0
:1008A000E30E05FCEF30904A832784049387F7FF1B
:1008B0002324F40483278404E34CF0FC9307F0FF23
:1008C0002324F404EF30906FEF30106C832744043E
:1008D000635AF00483270401638607049304040128
:1008E0006F000002832744049387F7FF2322F40458
:1008F000832744046358F0028327040163840702BA
:1009000013850400EF305017E30E05FCEF30104460
:10091000832744049387F7FF2322F40483274404A6
:10092000E34CF0FC9307F0FF2322F404032481003E
:100930008320C10083244100130101016F3010683E
:1009400063000508130101FF232481002322910085
:10095000130405002326110093840500EF30D062B4
:10096000832604048327C40303270400232C0402E2
:10097000B387F6021306F0FF2322C4042324E40005
:100980002324C404B386D740B307F7003307D70046
:100990002322F4002326E400639804028327040141
:1009A000639E0702EF3090618320C1000324810021
:1009B000832441001305100013010101678000002A
:1009C000737004306F00000013050401EFF01FD6B0
:1009D00013054402EFF09FD56FF0DFFC130504010F
:1009E000EF30900993071000E31EF5FAEFF05FBABD
:1009F0006FF05FFB63160500737004306F0000003A
:100A0000130101FE232A910023282101232631010D
:100A1000232E1100232C8100930906001389050061
:100A200093040500638E05083305B50213055505CB
:100A3000EF50803D13040500630C0508930745053E
:100A40002320F500232E940223202405EF30D053D9
:100A5000832604048327C403032704001306F0FF3E
:100A6000B387F602232C04022322C4042324E400C7
:100A70002324C40413050401B386D740B307F70049
:100A80003307D7002322F4002326E400EFF01FCA27
:100A900013054402EFF09FC9EF305052230834058C
:100AA000130504008320C101032481018324410133
:100AB000032901018329C10013010102678000009D
:100AC00013054005EF50403413040500631605007C
:100AD000737004306F000000232084006FF09FF6D5
:100AE00063160500737004306F0000006376B50074
:100AF000737004306F000000130101FF2324810094
:100B0000130620001384050093050000232611001E
:100B1000EFF05FEE630C0500232C85028320C100FB
:100B20000324810013010101678000007370043009
:100B30006F000000130101FB23261104232481040C
:100B40002322910423202105232E3103232C41034A
:100B5000232A510323286103232671032326C1007E
:100B600063060528638C052693072000639CF60026
:100B70000327C503930710006306F7007370043062
:100B80006F0000001389060093840500130405001C
:100B9000EF30D01F631A05008327C100638607006A
:100BA000737004306F000000EF30103E03278403A1
:100BB0008327C403130B0000930B20009309F0FF5D
:100BC000130A0401930A44026364F710630479234F
:100BD0008327C1006382073663160B00130581016A
:100BE000EF305004EF30903DEF20802FEF30D039C0
:100BF0008327440463943701232204048327840455
:100C00006394370123240404EF30503B9305C10063
:100C100013058101EF30100463160530EF30D03634
:100C2000032784038327C4036304F710EF301039CC
:100C3000EF309035832784046346F0026F00000391
:100C400013850A00EF30406363040500EF30101095
:100C5000832784049387F7FF2324F40483278404E1
:100C60006356F00083274402E39C07FC23243405E9
:100C7000EF30D034EF305031832744046346F00224
:100C80006F00000313050A00EF30005F63040500E6
:100C9000EF30D00B832744049387F7FF2322F4041B
:100CA000832744046356F00083270401E39C07FC78
:100CB00023223405EF309030EF200056130B100044
:100CC000EF30902C032784038327C403E370F7F0ED
:100CD0000326040463040612631A091E0325840014
:100CE00093850400EF50C0328327840083260404D8
:100CF00003274400B387D7002324F40063E4E710FC
:100D00008327840383260400032744029387170064
:100D10002324D400232CF40263000710130544029B
:100D2000EF308055930710006318F50E6F004014E4
:100D3000EF30D0288325C10013050A00EF30C0260C
:100D4000EF309024832784046346F0026F00000391
:100D500013850A00EF30405263040500EF30007F36
:100D6000832784049387F7FF2324F40483278404D0
:100D70006356F00083274402E39C07FC23243405D8
:100D8000EF30D023EF305020832744046346F00235
:100D90006F00000313050A00EF30004E63040500E6
:100DA000EF30C07A832744049387F7FF2322F404AB
:100DB000832744046356F00083270401E39C07FC67
:100DC00023223405EF30901FEF200045E31805EE95
:100DD000EFF00FFC130B10006FF09FEE832705045C
:100DE000E38407D8737004306F0000007370043020
:100DF0006F00000003260404631006088327040024
:100E0000638607048327840303274402938717001C
:100E1000232CF402E31407F0EF30501A13051000EE
:100E20008320C10403248104832441040329010491
:100E30008329C103032A8103832A4103032B01036E
:100E4000832BC102130101056780000003254400C4
:100E5000EF309006832784030327440223220400F3
:100E600093871700232CF402E31A07EAE30605FA36
:100E7000EFF00FF26FF05FFA0325C40093850400D2
:100E8000EF500019832704040327C40083260400BD
:100E9000B307F0403307F7002326E400637ED7044E
:100EA00003274400B307F7002326F40013072000AC
:100EB000832744026304E90403278403130717000C
:100EC000232CE402E38A07F46FF05FE50325C400F6
:100ED00093850400EF50C013832704040327C40044
:100EE00083260400B307F0403307F7002326E4000D
:100EF000E37ED7FA6FF0DFFA8327440203278403E7
:100F0000E30C07FA032784031307F7FF232CE402FB
:100F10000327840313071700232CE402E38E07EE54
:100F20006FF0DFDF13050400EFF05F92EF20C02EBB
:100F3000130500006FF0DFEEEF30500813050000DE
:100F40006FF01FEE130101FF2322910093040500AF
:100F5000130540052324810023261100EF40D06AA9
:100F600013040500630C0504232C05029307F0FF0E
:100F70002322F5041307100013050501232EE402B4
:100F80002324F40423220400232004002324040047
:100F9000232604002320040423089404EFF00FF90F
:100FA00013054402EFF08FF89306000013060000CB
:100FB0009305000013050400EFF0DFB713050400EC
:100FC0008320C10003248100832441001301010117
:100FD0006780000063040504130101FF23248100DE
:100FE00023229100232611002320210103294500FB
:100FF00013040500EF308058930400006304A90235
:101000008320C1000324810013850400032901000B
:1010100083244100130101016780000073700430D4
:101020006F0000008327C400930410009387F7FF2C
:101030002326F400E39607FC930600001306000045
:101040009305000013050400EFF0DFAE6FF05FFBC7
:10105000130101FC232E1102232C8102232A910269
:101060002328210323263103232441032326C100FF
:10107000630E050A930900006384051013890600B6
:101080009384050013040500130A05016F00800313
:10109000EF30C072EF30406F9305C100130581013E
:1010A000EF30403B63100506EF30006E03278403EA
:1010B0008327C403630CF702EF304070EF300070F9
:1010C00093091000EF30406C032784038327C40387
:1010D0006362F7068327C10063860702E39A09FA71
:1010E00013058101EF3000346FF09FFAEF30006D8F
:1010F0008325C10013050A00EF20106BEFF04FC9E4
:101100006FF0DFFBEF30806B8320C103032481038A
:1011100083244103032901038329C102032A810295
:101120001305000013010104678000007370043090
:101130006F000000032604046314060683270400DE
:1011400063880704832784030327440293871700D7
:10115000232CF40263100708EF3040668320C1039C
:101160000324810383244103032901038329C1024A
:10117000032A810213051000130101046780000097
:1011800083270504E38C07EE737004306F000000C2
:1011900003254400EF304052232204006FF09FFAF1
:1011A000631609040325840093850400EF4050660C
:1011B000832784008326040403274400B387D700D1
:1011C0002324F400E3E0E7F8832704002324F40059
:1011D0006FF05FF713054402EF30000A9307100029
:1011E000E31CF5F6EFF0CFBA6FF01FF70325C4004C
:1011F00093850400EF40D061832704040327C400D3
:1012000083260400B307F0403307F7002326E400E9
:101210006378D70003274400B307F7002326F400C0
:1012200093072000E310F9F283278403E38C07F08F
:10123000832784039387F7FF232CF4026FF09FF03A
:10124000130101FC232E1102232C8102232A910277
:101250002328210323263103232441032326C1000D
:101260006308051493040000638C0512938906003B
:101270001389050013040500130A45026F000001DD
:10128000EF30C053EF30805393041000EF30C04F65
:1012900083278403639E07088327C100638C0704A8
:1012A00063840404EF308051EF30004E9305C10099
:1012B00013058101EF30001A631E0502EF30C04CA8
:1012C00083278403E39E07FAEF30404F832704000F
:1012D000638607048325C10013050A00EF20D04C64
:1012E000EFF00FAB6FF01FFA13058101EF308013A1
:1012F0006FF05FFBEF30804C8320C1030324810338
:1013000083244103032901038329C102032A8102A3
:10131000130500001301010467800000EF30C04690
:1013200003254400EF304029EF3040496FF09FFA29
:10133000032604048324C400630406020327440034
:10134000B387C4002326F40063E6E7008327040084
:101350002326F4008325C40013050900EF40504BF9
:10136000639C090483278403032704009387F7FF02
:10137000232CF40263160700EF30804B2322A400D5
:10138000832704016380070413050401EF20D06E56
:10139000930710006318F502EFF08F9F6F00800233
:1013A00083270504E38407EC737004306F000000AA
:1013B000737004306F0000008327440223269400DA
:1013C00063960702EF30803F8320C103032481032B
:1013D00083244103032901038329C102032A8102D3
:1013E0001305100013010104678000001305440277
:1013F000EF209068E30805FC6FF01FFA6302050A0E
:1014000063880508130101FE232C8100232A910023
:101410002328210123244101232E110023263101F9
:10142000930720009384060013090600138A050021
:1014300013040500639CF6000327C50393071000FF
:101440006302F70A737004306F000000EFF08FA89A
:10145000032784038327C403930905006366F70405
:101460009304000013850900EFF04FA68320C1010B
:101470000324810113850400032901018324410110
:101480008329C100032A8100130101026780000043
:1014900083270504E38807F6737004306F000000AB
:1014A000737004306F00000003260404631E060CF2
:1014B0008327040063860712832784031307F0FF42
:1014C00093871700232CF402832784046388E70E94
:1014D0008327840493041000938717002324F404C3
:1014E0006FF05FF8EFF00F9F032784038327C40397
:1014F000930905006360F70603260404E30A06FA6D
:101500000325C40093050A00EF40903083270404AC
:101510000327C40083260400B307F0403307F70015
:101520002326E4006378D70003274400B307F700BD
:101530002326F40093072000E390F4F88327840324
:10154000E38C07F6832784039387F7FF232CF402A9
:101550006FF09FF603260404E30C06F40325C40091
:1015600093050A00EF40D02A832704040327C40010
:1015700083260400B307F0403307F7002326E40076
:10158000E364D7FA6FF09FFBE39C04F60325840025
:1015900093050A00EF40D0278327840083260404A4
:1015A00003274400B387D7002324F400E3E6E7F0E1
:1015B000832704002324F4006FF01FF083274402E4
:1015C00093041000E38007EA13054402EF20D04A99
:1015D000E30A05E8E30809E8232099006FF09FE893
:1015E00003254400EF30400D232204006FF0DFECB0
:1015F0006302050A832705046386070073700430BD
:101600006F00000083270500638A0708130101FEAD
:10161000232C8100232A9100130405002328210193
:1016200023263101232E110013890500EFF08F8A44
:10163000032784038327C403930905009304000050
:101640006376F702832784031307F0FF938717005D
:10165000232CF40283278404638AE7048327840409
:1016600093041000938717002324F40413850900C2
:10167000EFF0CF858320C10103248101138504008D
:1016800003290101832441018329C10013010102BF
:1016900067800000737004306F00000083274500EE
:1016A000E38607F6737004306F000000832744025E
:1016B00063960700930410006FF05FFB130544026C
:1016C000EF20903BE30805FEE30609FE93071000B8
:1016D0002320F9006FF01FFE130101FC232E1102DD
:1016E000232C8102232A910223282103232631035C
:1016F00023244103232251032326C1006306052826
:10170000638C0526938A060093890500130405005F
:10171000EF20D067631A05008327C10063860700A6
:10172000737004306F000000EF30000683278403DD
:101730006394071C8327C100638007101305810190
:10174000EF20504E9304F0FF13094402130A0401E2
:10175000EF30C006EF10C078EF3000038327440459
:1017600063949700232204048327840463949700DE
:1017700023240404EF3080049305C1001305810184
:10178000EF20504D63100524EF30000083278403C1
:10179000638A070AEF308002EF20107F83278404DA
:1017A0006346F0026F00000313050900EF20D02C00
:1017B00063040500EF209059832784049387F7FF83
:1017C0002324F404832784046356F000832744020F
:1017D000E39C07FC23249404EF20507EEF20D07A72
:1017E000832744046346F0026F00000313050A00D8
:1017F000EF20902863040500EF2050558327440410
:101800009387F7FF2322F404832744046356F000F0
:1018100083270401E39C07FC23229404EF20107A21
:10182000EF10901FEF205076832784036396070CF8
:101830008327C100E39E07F0EF20507813050000D6
:101840006F00800FEF2090778327040063880710D4
:101850008325C10013050900EF200075EF20D07229
:10186000832784046346F0026F0000031305090018
:10187000EF20902063040500EF20504D832784045F
:101880009387F7FF2324F404832784046356F0002E
:1018900083274402E39C07FC23249404EF20107266
:1018A000EF20906E832744046346F0026F0000032C
:1018B00013050A00EF20501C63040500EF201049B7
:1018C000832744049387F7FF2322F40483274404E7
:1018D0006356F00083270401E39C07FC2322940451
:1018E000EF20D06DEF10501363040508EF20D0698E
:1018F00083278403E38E07F2938509001305040010
:101900008324C400EFE05FF163940A088327840313
:10191000032704009387F7FF232CF40263160700C4
:10192000EF2010712322A40083270401639207088B
:10193000EF20D068130510008320C1030324810326
:1019400083244103032901038329C102032A81025D
:10195000832A41021301010467800000EF20D06256
:1019600003254400EF205045EF2050656FF05FEEF7
:10197000EFE01FC26FF09FF783270504E38407D8C9
:10198000737004306F000000737004306F0000004B
:101990008327440223269400E38C07F813054402AE
:1019A000EF20900DE30605F8EFE09FBE6FF05FF8C3
:1019B00013050401EF20500C93071000E31AF5F60D
:1019C0006FF09FFE13050400EFE05FE8EF10D00416
:1019D000130500006FF05FF663000506130101FFB9
:1019E000232481002320210123261100232291009A
:1019F000832445001389050013040500EF201038E7
:101A00006380A404930600001306090093050000F8
:101A100013050400EFF05FCC93071000630CF50290
:101A20008320C10003248100832441000329010095
:101A30001301010167800000737004306F00000023
:101A40008327C40013051000938717002326F40092
:101A50006FF01FFD8327C400938717002326F4002F
:101A60006FF01FFC630805066386050C130101FE79
:101A7000232C8100232A91002328210123263101D0
:101A80002324410113040500232E1100130906002D
:101A900093890500EFE01FC483278403130A050020
:101AA00093040000639C070213050A00EFE01FC2C5
:101AB0008320C1010324810113850400032901014E
:101AC000832441018329C100032A810013010102FB
:101AD00067800000737004306F0000000326040468
:101AE000630406028325C40083274400B385C50030
:101AF0002326B40063E6F500832504002326B40002
:101B000013850900EF40C050832784031307F0FFBB
:101B10009387F7FF232CF402832744046384E702AE
:101B20008327440493041000938717002322F404AE
:101B30006FF09FF783270504E38A07F27370043080
:101B40006F000000832704016396070093041000D0
:101B50006FF09FF513050401EF200072E30805FE06
:101B6000E30609FE930710002320F9006FF01FFE23
:101B70006306050883270504638A0508638407084C
:101B8000130101FE232C8100232A91002328210127
:101B90002324410113040500232E110023263101C3
:101BA000138A0500EFE01FB38327840313090500A0
:101BB00093040000638E07008329C40093050A0084
:101BC00013050400EFE05FC59304100023263401E1
:101BD00013050900EFE09FAF8320C10103248101B9
:101BE0001385040003290101832441018329C100D5
:101BF000032A810013010102678000007370043022
:101C00006F000000737004306F000000E38C07FE6B
:101C1000737004306F0000006316050073700430A9
:101C20006F000000130101FF23248100130405004D
:101C300023261100EF20503503248403EF201038B1
:101C40008320C10013050400032481001301010156
:101C50006780000063160500737004306F00000099
:101C6000130101FF23261100232481001304050022
:101C7000EF209031832784030324C4033304F4400A
:101C8000EF20D033130504008320C100032481001A
:101C90001301010167800000630605000325850329
:101CA00067800000737004306F0000006308050453
:101CB00097870300938707AD03A747006304E504F4
:101CC00003A7C7006302E50803A74701630AE50607
:101CD00003A7C7016302E50603A74702630AE504F9
:101CE00003A7C7026302E50403A74703630AE502EB
:101CF00003A7C7036302E5026F4000297370043035
:101D00006F0000001307000013173700B387E700C8
:101D100023A007006F404027130770006FF0DFFE1D
:101D2000130760006FF05FFE130750006FF0DFFDD8
:101D3000130740006FF05FFD130730006FF0DFFC0A
:101D4000130720006FF05FFC130710006FF0DFFB3C
:101D50000325C504678000002326B50467800000C2
:101D6000034505056780000063080500032585031A
:101D70001335150067800000737004306F00000099
:101D8000630C0500832785030325C5033305F54050
:101D90001335150067800000737004306F00000079
:101DA000978703009387079E03A707006300070434
:101DB00003A787006308070403A707016308070454
:101DC00003A787016308070403A707026308070442
:101DD00003A787026308070403A70703630C07042C
:101DE00003A787036304070467800000130700004C
:101DF00013173700B387E70023A0B70023A2A7007B
:101E000067800000130710006FF09FFE130720008B
:101E10006FF01FFE130730006FF09FFD13074000A7
:101E20006FF01FFD130750006FF09FFC1307700049
:101E30006FF01FFC130760006FF09FFB9787030094
:101E40009387479403A747006300E50403A7C700EF
:101E50006306E50403A747016306E50403A7C7017A
:101E60006306E50403A747026306E50403A7C70268
:101E70006306E50403A74703630AE50403A7C70352
:101E80006302A704678000001307000013173700E0
:101E9000B387E70023A00700678000001307100046
:101EA0006FF0DFFE130720006FF05FFE13073000B6
:101EB0006FF0DFFD130740006FF05FFD1307500068
:101EC0006FF0DFFC130770006FF05FFC130760001A
:101ED0006FF0DFFB130101FF232481002322910017
:101EE00023202101130405002326110093840500FB
:101EF00013090600EF205009032744049307F0FF5D
:101F00006314F70023220404032784049307F0FFDB
:101F10006314F70023240404EF20500A832784036A
:101F2000639A070013060900938504001305440211
:101F3000EF20C023EF20500583278404635AF00468
:101F40008327440263860704930444026F0000025F
:101F5000832784049387F7FF2324F40483278404CE
:101F60006358F00283274402638407021385040048
:101F7000EF208030E30E05FCEF20405D83278404D2
:101F80009387F7FF2324F40483278404E34CF0FCB5
:101F90009307F0FF2324F404EF205002EF20C07ECB
:101FA00083274404635AF0048327040163860704EB
:101FB000930404016F000002832744049387F7FF12
:101FC0002322F404832744046358F0028327040186
:101FD0006384070213850400EF20002AE30E05FC4A
:101FE000EF20C056832744049387F7FF2322F4048D
:101FF00083274404E34CF0FC9307F0FF2322F4040E
:10200000032481008320C1008324410003290100AF
:10201000130101016F20807A63040504130101FD9F
:10202000232E3101232C410123261102138A07009C
:10203000232481022322910223202103232A5101F8
:102040002328610123267101232481019307900035
:102050009309070063FAE700737004306F00000013
:10206000737004306F000000930A0500938405002C
:1020700013090600938B0600130B08006304082C59
:1020800013050006EF305058130405006304052AB9
:102090001319290023286503130609009305500A24
:1020A00013050B00EF40C00803C704008327040397
:1020B0001309C9FF230AE40203C704003389270177
:1020C0001379C9FF6306070E83C71400A30AF4023D
:1020D00083C71400638E070C83C72400230BF4020C
:1020E00083C724006386070C83C73400A30BF40264
:1020F00083C73400638E070A83C74400230CF402AD
:1021000083C744006386070A83C75400A30CF40204
:1021100083C75400638E070883C76400230DF4024D
:1021200083C764006386070883C77400A30DF402A5
:1021300083C77400638E070683C78400230EF402EE
:1021400083C784006386070683C79400A30EF40246
:1021500083C79400638E070483C7A400230FF4028F
:1021600083C7A4006386070483C7B400A30FF402E7
:1021700083C7B400638E070283C7C4002300F4043E
:1021800083C7C4006386070283C7D400A300F40496
:1021900083C7D400638E070083C7E4002301F404DF
:1021A00083C7E4006386070083C7F400A301F40437
:1021B000130B440013050B00A3010404232634036E
:1021C00023283405232A0404EFE04FD813058401A3
:1021D000EFE0CFD79307A000B3873741232C040447
:1021E00023288400232CF4002322840223220404C5
:1021F000232E040413860B0093850A00130509009F
:10220000EFE00FCE2320A40063040A0023208A00FD
:102210007370043017E901001309C92983270900E5
:1022200097E401009384C42A638C070003A7040089
:1022300083A7040083274704938717002322F7040A
:1022400017E701001307C7278327070093871700A5
:1022500097E6010023A6F62683A7040063800710F3
:102260008327090017EA0100130A8A35639C0700D7
:1022700083A7040083A7C70263E6F90097E701007C
:1022800023A8872497E701009387C72103A70700A6
:1022900097E60100938646228327C40283A60600A0
:1022A0001307170017E60100232EE61E2324E4047B
:1022B00063F6F60017E701002320F720130740011B
:1022C000B387E70293050B003305FA00EFE08FC8F0
:1022D000832709006388070083A7040083A74704B6
:1022E000639E07088327090013041000638A070010
:1022F00083A7040083A7C70263F43701EFE04FA967
:10230000130504008320C1020324810283244102B7
:10231000032901028329C101032A8101832A410182
:10232000032B0101832BC100032C81001301010346
:102330006780000013050B00EF3010451304F0FF19
:102340006FF01FFC13152600EF30102C130B050047
:10235000E31805D21304F0FF6FF09FFA97E701002E
:1023600023A887160327070093071000630AF702C4
:1023700017EA0100130ACA246FF0DFF003A7040074
:1023800083A60400832747049387F7FF2322F704DB
:1023900083A74604E39807F4736004306FF09FF45A
:1023A000930A000017EA0100130A8A21130C400166
:1023B000930BA00033858A03938A1A003305AA0081
:1023C000EFE0CFB6E3987AFF97EB0100938BCB2B2E
:1023D00013850B00EFE08FB597EA0100938A0A2C72
:1023E00013850A00EFE08FB417E501001305452CB3
:1023F000EFE0CFB317E501001305C52CEFE00FB3F5
:1024000017E501001305452DEFE04FB297E70100F6
:1024100023AE770B97E7010023A8570B6FF09FE6D9
:10242000130101FF232481002326110023229100A0
:1024300023202101130405007370043097E4010088
:102440009384440783A70400639E07106318040065
:1024500097E701009387C70703A407001309440007
:1024600013050900EFE04FB7832784026386070056
:1024700013058401EFE04FB69305090017E501004D
:1024800013054524EFE00FAD97E70100938787031D
:1024900003A7070097E701009387C70083A70700FA
:1024A0001307170097E6010023AEE60003A7040018
:1024B0009387170097E6010023A6F6FE630C07003A
:1024C00097E701009387C70003A707000327470486
:1024D000631C070E83A70400638A070697E70100C1
:1024E000938707FF03A70700630287107370043008
:1024F00003A704006318070817E70100130707FD87
:102500008326070083A606006392060A1307F0FFDE
:1025100097E6010023A6E6F803A704006308070274
:1025200003A70700032747046302070203A7070066
:1025300083A60700832747049387F7FF2322F70426
:1025400083A7460463940700736004308320C100AE
:1025500003248100832441000329010013010101A8
:102560006780000097E70100938787F603A70700BD
:1025700083A7070083274704938717002322F704C4
:102580006FF0DFEC83A6070003A7070003A746044C
:102590001307170023A2E60417E70100130707F348
:1025A0008326070083A60600E38206F603270700BA
:1025B0000327C7000327C7000327470097E601004A
:1025C00023A0E6EE6FF05FF503A7070083A60700E0
:1025D000832747049387F7FF2322F70483A7460442
:1025E000E39A07EE736004306FF0DFEE97E70100C7
:1025F0009387C7EA83A707006386070073700430D8
:102600006F000000032481008320C1008324410067
:1026100003290100130101016FD09FF76304050C2A
:1026200017E701001307C7EA832607009307000096
:102630006386A60A130101FF2326110023248100CB
:10264000232291007370043097E60100938686E69A
:1026500083A70600638C0700032607008327070073
:1026600083274604938717002322F60483A70600D6
:1026700093040500032445016388070083270700AE
:1026800083A747046394070697E70100938707E44D
:1026900083A70700638C870697E701009387C7E24B
:1026A00083A707006384870697E701009387C70223
:1026B0006306F40497E701009387C700630CF402F4
:1026C000930710008320C10003248100832441006C
:1026D00013850700130101016780000013850700BF
:1026E00067800000737004306F000000EF60002B03
:1026F0006FF09FF9930740006FF0DFFC83A784021F
:1027000093B71700938727006FF0DFFB9307200034
:102710006FF05FFB7370043097E70100938787D9F0
:1027200003A70700631607026304050483A70700D5
:102730000325C502638C070097E70100938747D9FB
:1027400003A7070003274704631C070267800000F4
:1027500017E701001307C7D78326070003270700E1
:1027600003A746041307170023A2E604E31005FCA1
:1027700017E701001307C7D5032507006FF01FFBFC
:1027800003A7070083A60700832747049387F7FF63
:102790002322F70483A74604E39A07FA7360043000
:1027A00067800000130101FF23248100130405004A
:1027B00023261100EFD01FF26318040097E70100F1
:1027C000938707D103A407000324C402EFD01FF0AE
:1027D0008320C100130504000324810013010101BB
:1027E000678000009307900063F6B70073700430B1
:1027F0006F000000130101FE232C8100232E110025
:10280000232A910023282101232631012324410179
:10281000130405007370043017E90100130989C916
:1028200083270900639207106300041283270405BD
:10283000638EF50A17E70100130787C963F0B70233
:1028400083260700638E8612032707008324C702AE
:10285000B3B4950093C414006F00000183240700F3
:10286000B384844093B414000327C4026386E70E44
:10287000832784012328B40463C807009307A000BA
:10288000B385B740232CB40093172700B387E70024
:102890000327440197E90100938989D29397270080
:1028A000B387F9006310F704130A440013050A0004
:1028B000EFD09FF217E70100130707C08327C40278
:1028C000032707006376F70017E701002326F7BE0A
:1028D00013074001B387E70293050A003385F90027
:1028E000EFD05FE763840400EFD09FCA832709001D
:1028F000638C070097E70100938787BD83A70700D4
:1029000083A74704639E07048320C1010324810138
:1029100083244101032901018329C100032A810085
:10292000130101026780000097E70100938747BA0F
:1029300003A7070083A7070083274704938717008F
:102940002322F704E31404EE97E70100938747B8C6
:1029500003A407006FF09FED2326B4026FF05FF130
:10296000032481018320C101832441010329010142
:102970008329C100032A8100130101026F60000254
:10298000930400006FF05FEE630A0508130101FE77
:10299000232A910097E40100938484B383A7040061
:1029A000232E1100232C810023282101232631010D
:1029B0006388A7047370043017E90100130989AF15
:1029C00083270900638C070003A7040083A7040082
:1029D00083274704938717002322F7040327450121
:1029E00097E70100938747CF630EF702832709001B
:1029F0006388070083A7040083A74704639E070832
:102A00008320C101032481018324410103290101A1
:102A10008329C10013010102678000007370043034
:102A20006F0000008327850217E70100130747C8DE
:102A3000E38EE7FAE39C07FA9309450013040500C7
:102A400013850900EFD05FD917E701001307C7A668
:102A50008327C402032707006376F70017E7010006
:102A6000232CF7A413074001B387E70217E5010001
:102A7000130505B5938509003305F500EFD09FCD0B
:102A800083A704000327C40283A7C702E360F7F605
:102A9000EFD01FB06FF09FF5032481018320C101A7
:102AA00083244101032901018329C100130101028B
:102AB0006F50D06E63020506130101FE232C8100C6
:102AC000232A91002328210113040500232E11003D
:102AD00023263101EFD01FC00327440197E70100EF
:102AE000938787BF1309050093040000630AF70268
:102AF00013050900EFD09FBD8320C101032481018C
:102B00001385040003290101832441018329C100A5
:102B10001301010267800000737004306F00000031
:102B20008327840217E50100130585B8E382A7FC1B
:102B3000E39007FC97E701009387479683A7070078
:102B40006394070697E701009387879883A7070098
:102B50008324C4029309440083A7C7021385090094
:102B6000B3B4F400EFD05FC717E701001307C794B1
:102B70008327C4020327070093C414006376F70079
:102B800017E70100232AF79213074001B387E702F2
:102B900017E501001305C5A2938509003305F5006B
:102BA000EFD05FBB6FF0DFF493058401EFD09FBAE5
:102BB0006FF01FF4130101FE37150000232E1100E2
:102BC000232C8100232A910023282101232631016F
:102BD000232441012322510123206101EF30C0222F
:102BE000630805229304050013050006EF30C02199
:102BF0001304050063040526371600009305500AE8
:102C00002328950213850400EF30805283240403A7
:102C1000B71700009387C7FFB384F400B7474C454C
:102C200093879744130A4400232AF40213050A00E9
:102C3000230C0402A3010404232604022328040411
:102C4000232A0404EFD09FB013058401EFD01FB0F6
:102C50009307A000232C040493F4C4FF23288400CA
:102C6000232CF4002322840223220404232E0404B0
:102C700013060000971500009385C5EA138504002C
:102C8000EFD01FA62320A4007370043017E90100C1
:102C9000130949828327090097E401009384448340
:102CA000638C070003A7040083A70400832747045D
:102CB000938717002322F70417E7010013074780C3
:102CC000832707009387170097D6010023AAF67E73
:102CD00083A704006388070A8327090097E9010096
:102CE0009389098E639C070083A7040083A7C7020A
:102CF0006396070097D7010023AC877C97D7010024
:102D00009387477A03A7070097D601009386C67A70
:102D10008327C40283A606001307170017D60100F5
:102D20002322E6782324E40463F6F60017D7010093
:102D30002324F778139527003305F5001315250094
:102D400093050A003385A900EFD0DFA0832709008F
:102D50006388070083A7040083A74704639E070CCA
:102D6000832709006384070083A70400EF2050062F
:102D700093071000630AF510631C05087370043094
:102D80006F00000097D7010023A487740327070072
:102D90009307100097E9010093898982E310F7F601
:102DA000938A090017EB0100130B0B8E13850A00A1
:102DB000938A4A01EFD09F97E31A5BFF17E5010062
:102DC0001305858CEFD09F9697EA0100938A0A8DB0
:102DD00013850A00EFD09F9517E501001305458D77
:102DE000EFD0DF9417E501001305C58DEFD01F94D8
:102DF00017E501001305458EEFD05F9397D70100CB
:102E000023A6676D97D7010023A0576D6FF01FEFC2
:102E10008320C1010324810183244101032901018D
:102E20008329C100032A8100832A4100032B01006A
:102E3000130101026780000003A7040083A60400B9
:102E4000832747049387F7FF2322F70483A74604C9
:102E5000E39807F0736004306FF09FF00324810162
:102E60008320C101032901018329C100032A8100B4
:102E7000832A4100032B01001385040083244101B0
:102E8000130101026F304010737004309307F0FF9C
:102E900017D701002326F7600324810197D701008B
:102EA00023AAA7608320C1018324410103290101D2
:102EB0008329C100032A8100832A4100032B0100DA
:102EC00097D7010023AC075E130101026FD08FD1A9
:102ED0007370043097D7010023AE075C6FD0CFE248
:102EE00017D701001307875B832707009387170015
:102EF0002320F700678000007370043097D701002B
:102F00009387475B03A707006318070217D70100E1
:102F10001307C75A0325070083A70700638C070020
:102F200097D701009387C75A03A7070003274704D1
:102F3000631407026780000017D701001307475981
:102F4000832607000327070003A74604130717007B
:102F500023A2E6046FF09FFB03A7070083A60700E8
:102F6000832747049387F7FF2322F70483A74604A8
:102F7000E39207FC7360043067800000130101FFD7
:102F80002326110023248100EFD0CFF497D701002E
:102F90009387C75203A40700EFD04FF38320C100EB
:102FA0001305040003248100130101016780000060
:102FB00097D701009387C75003A5070067800000DB
:102FC000130101FD232611022324810223229102F1
:102FD00023202103232E3101232C4101232A5101D7
:102FE000232861012326710197D701009387074B9E
:102FF00083A70700639A070617D701001307074C3A
:10300000832707009387170097D6010023A8F64A65
:10301000832A0700638A0A0A97D7010093874748E3
:1030200083A707009304000063FEFA0A97D9010002
:103030009389095917DA0100130A8A4983270A007C
:103040009306100003A7C70293172700B387E70072
:1030500093972700B389F90083A7090063F4F60268
:10306000930410006F00000297D701009387474434
:1030700083A70700930400009387170017D7010068
:103080002328F74297D701009387474283A7070079
:1030900063840700930410008320C102032481028B
:1030A0001385040003290102832441028329C101FD
:1030B000032A8101832A4101032B0101832BC100D3
:1030C000130101036780000017D4010013040440BA
:1030D0008327040083A707006388070C73700430FC
:1030E0006F00000017D401001304443E97D901007B
:1030F0009389094D17DA0100130A8A3D17DB010095
:10310000130B8B3B8327040083A70700638007080A
:103110008327040083A7C70003A9C70083274900AA
:10312000930B490013850B0063EAFA06EFD0CFEA50
:10313000832789021305890163840700EFD0CFE953
:103140008327C90203270B0093850B0013952700E3
:103150003305F500131525003385A9006376F700C4
:1031600017D70100232AF734EFD0CFDE83270A00D8
:103170000327C90283A7C702E366F7F88327040081
:103180009304100083A70700E39407F89307F0FF68
:1031900017D701002326F7306FF05FEA17D7010039
:1031A0002320F7306FF09FE917D701001307C731CD
:1031B000832704000327070097D6010023A8E630E1
:1031C00017D701002322F73097D701009387C72D27
:1031D00083A707009387170017D701002326F72C32
:1031E0008327040083A70700639A07009307F0FF73
:1031F00017D701002326F72A6FF01FE28327040068
:1032000083A7C70083A7C70083A7470017D701007C
:103210002328F7286FF05FE097D7010093870728EE
:1032200003A7070063160700737004306F000000E7
:10323000130101FE232E1100232C8100232A91006B
:103240002328210123263101232441012322510176
:10325000232061017370043097D401009384842586
:1032600003A704006310071203A707001307F7FF63
:1032700097D6010023A4E62283A70700639E070ACE
:1032800097D701009387C72383A707006386070AA0
:1032900097DA0100938ACA3217DA0100130ACA21A9
:1032A00017D901001309C922930910006F00C0014A
:1032B0003385EA00EFD00FCA832709000327C40231
:1032C00083A7C7026374F70683A70A0F6380070EFC
:1032D00083A7CA0F03A4C70013058401EFD0CFCF83
:1032E000130B440013050B00EFD00FCF8327C4024C
:1032F00083260A0093050B00139527003305F5007C
:1033000013152500130705003385AA00E3F2F6FA2A
:1033100017D701002322F71AEFD0CFC38327090064
:103320000327C40283A7C702E360F7FA97D7010017
:1033300023AE37176FF05FF91304000083A7040072
:10334000638C070097D701009387871883A707002E
:1033500083A7470463980704130504008320C10171
:103360000324810183244101032901018329C10030
:10337000032A8100832A4100032B0100130101026B
:103380006780000017D70100130787148326070002
:103390000327070003A746041307170023A2E60428
:1033A0006FF09FECEF50805F6FF01FFB17D40100B0
:1033B0001304041083270400638C0702832704008E
:1033C0001309100063860702EFF09FBF6306050034
:1033D00097D7010023AC270D832704009387F7FFBD
:1033E00017D701002326F70C83270400E39E07FC70
:1033F00097D701009387870B03A707009307100057
:10340000E31CF7F2EFD0CF98130410006FF01FF316
:103410006304050263960500737004306F000000BA
:1034200017D701001307870783270700638A070060
:10343000737004306F000000737004306F00000080
:10344000130101FF23248100232611008326070096
:10345000032705009386160017D601002320D60403
:1034600097D601009386860583A606003304B7002D
:103470002320850063F0E6046372E40263F08602B1
:1034800097D701009387C70403A5070013054500DC
:10349000EFD08FB413050400EF50C047EFF0DFD733
:1034A000630E05008320C100032481001301010184
:1034B00067800000E366E4FC6FF05FFC032481009A
:1034C0008320C100130101016FD08F8C630E0500B2
:1034D00017D70100130787FC8327070063880700BD
:1034E000737004306F0000006FD08F8A130101FFEA
:1034F00023261100232481000327070093070500DA
:103500001307170097D6010023AAE6F897D6010003
:10351000938606FC17D70100130747FA0327070015
:1035200003A506003304F70013054500EFD0CFAA2A
:1035300013050400EF50003EEFF01FCE631A0500A4
:10354000032481008320C100130101016FD04F8447
:103550008320C10003248100130101016780000062
:10356000130101FF232481002326110097D70100B6
:103570009387C7F283A707001304000093871700FF
:1035800017D70100232CF7F097D70100938747F353
:1035900083A7070063EEF51417DE0100130E0E0E6D
:1035A00097D2010093820201130400001307000068
:1035B000930F10001303500A6F00C000130ECEFECD
:1035C0006384C20F83278EFF93060700E38807FEFC
:1035D0008327CEFF83A74700232EFEFE6386C713F3
:1035E00003AFC70083A747003307E500930E000031
:1035F000232EFEFE6380C70983A8C7009387480374
:10360000232017012322F70083A788042326F7012C
:103610002324F70083A7C8022328F70083A70805FF
:10362000232C0700232AF70003A808038347080078
:1036300063986704930708009387170083C6070001
:10364000B3850741E38A66FE93D52500939505016E
:1036500093D50501231EB700938E1E0013070702A2
:10366000630A1F038327CEFF83A74700232EFEFE96
:10367000E394C7F983274E00232EFEFE6FF0DFF799
:1036800093050000231EB700938E1E001307070248
:10369000E31A1FFD3304D40113175400130ECEFE9A
:1036A00093060700E390C2F397D70100938707E2E0
:1036B00003AE070083270E006396071297D7010019
:1036C000938787E003AE070083270E00639A071CE9
:1036D00017DE0100130ECEEE83274E10639C070207
:1036E00083278E11639C07266304060023200600AF
:1036F000EFF09FB2130504008320C1000324810072
:10370000130101016780000083274E00232EFEFE77
:103710006FF01FED83278E1017DF0100130F0FFBD3
:1037200083A7470017D701002320F7FA6386E73DF8
:1037300083A2C70083A74700B306D500930E0000FD
:1037400017D701002322F7F8930F40001303500A04
:103750006382E70983A8C7009387480323A0160163
:1037600023A2F60083A7880423A6F60123A4F6006B
:1037700083A7C80223A8F60083A7080523AC060088
:1037800023AAF60003A8080383470800639A673258
:10379000930708009387170003C70700B385074105
:1037A000E30A67FE93D725009397070193D7070194
:1037B000239EF600938E1E0093860602638C1231C0
:1037C00083278E1083A7470017D70100232EF7EE1B
:1037D000E392E7F983270E1117D701002326F7EEAE
:1037E0006FF05FF783274E00130F8E0083A647000C
:1037F0002322DE006380E633B307E50003A746001B
:1038000083A2C600930E00002322EE00930F200037
:103810001303500A6300EF088328C7001387480387
:1038200023A0170123A2E70003A7880423A6F7011A
:1038300023A4E70003A7C80223A8E70003A70805FD
:1038400023AC070023AAE70003A8080303470800E6
:10385000631E67221307080013071700834607003B
:10386000B3050741E38A66FE13D725001317070146
:1038700013570701239EE700938E1E0093870702CC
:103880006380122383264E0003A746002322EE0006
:10389000E314EFF80327CE002322EE006FF0DFF7EA
:1038A00083274E00130F8E0083A747002322FE00BC
:1038B000638CE72583A2C70083A74700B306D50022
:1038C000930E00002322FE00930F20001303500AE2
:1038D0006300FF0883A8C7009387480323A016014D
:1038E00023A2F60083A7880423A6F60123A4F600EA
:1038F00083A7C80223A8F60083A7080523AC060007
:1039000023AAF60003A808038347080063986714F6
:10391000930708009387170003C70700B385074183
:10392000E30A67FE93D725009397070193D7070112
:10393000239EF600938E1E0093860602638A12135E
:1039400083274E0083A747002322FE00E314FFF8DD
:103950008327CE002322FE006FF0DFF78327CE11EE
:1039600097DE0100938ECED783A7470017D70100BB
:103970002326F7D6638AD71783AFC70083A74700EC
:103980003307D5001303000097D6010023A8F6D40F
:10399000130F3000930220009308500A6388D70960
:1039A00003A5C700930745032320A7002322F700A0
:1039B000832785042326E7012324F7008327C502F4
:1039C0002328F700832785026384070023265700F6
:1039D00083270505232C0700232AF7000328050366
:1039E00083470800639C1705930708009387170017
:1039F00083C60700B3850741E38A16FF93D72500E6
:103A00009397070193D70701231EF70013031300B1
:103A100013070702638EAF028327CE1183A74700E7
:103A200097D6010023ACF6CAE39CD7F783274E1242
:103A300097D6010023A4F6CA6FF09FF69307000003
:103A4000231EF7001303130013070702E396AFFCCE
:103A500033046400E31C06C86FF09FC9930700009D
:103A6000239EF600938E1E0093860602E39A12EDC3
:103A700017DE0100130ECEB483274E103304D40199
:103A800093165400E38E07C46FF0DFC813070000DD
:103A9000239EE700938E1E0093870702E39412DFB4
:103AA00097D70100938747A203AE07003304D401E0
:103AB0009316540083270E00E38C07C06FF05FDE7F
:103AC00093070000239EF600938E1E009386060245
:103AD000E39812CF83278E113304D4019316540038
:103AE000E38407C06FF09FE783274E1217D70100CA
:103AF0002326F7BE6FF05FE883270E1117D701006A
:103B00002324F7BC6FF0DFC28327CE002322FE0000
:103B10006FF05FDA8326CE002322DE006FF0DFCD68
:103B2000130101FD2322910223202103232E3101C1
:103B3000232C4101232A51012328610123267101ED
:103B4000232611022324810297D901009389099524
:103B500017D901001309C9A617DA0100130A8A95BB
:103B600097DA0100938ACA9697DB0100938B4B95F5
:103B700097D4010093840495130B10006F0000028A
:103B800083A70900032449109387170017D7010062
:103B90002326F790EFF04FE8631E040083A704008C
:103BA000E39007FE83270900E37AFBFEEFC05F9EE8
:103BB0006FF0DFFE7370043083270A00639E0704F2
:103BC0008327091103A4C70013054400EFC0DFC019
:103BD00083A70B009387F7FF17D701002322F78EE7
:103BE00083A704009387F7FF17D70100232CF78CD6
:103BF00083270A006388070083A70A0083A7470476
:103C00006398070203250403EF200038130504001E
:103C1000EF2080376FF09FF803A70A0083A70A0000
:103C200083274704938717002322F7046FF05FF977
:103C300003A70A0083A60A00832747049387F7FF98
:103C40002322F70483A74604E39E07FA7360043037
:103C50006FF05FFB97D701009387478483A7070026
:103C60006396070E130101FF2326110097D7010069
:103C700023AE078217D70100130787858327070024
:103C8000B7A6A5A59386565A83A7070383A5070061
:103C9000639ED50003A64700631AB60083A687007B
:103CA0006396C60083A7C700638AD7000325070071
:103CB0008325070093854503EF30807697C6010082
:103CC0009386867F03A6060017D701001307478F48
:103CD0006F00000283A706006382070883A706001F
:103CE0009387F7FF17C601002328F67C03A606007A
:103CF00093172600B387C70093972700B307F700F1
:103D000083A70700E38807FC03A606009317260095
:103D1000B387C70093972700B305F70083A6450034
:103D200093878700B307F70083A6460023A2D50038
:103D3000638AF60283A7C6008320C10017C701006B
:103D40002328F77813010101678000009307100012
:103D500017C70100232CF7746780000073700430CC
:103D60006F000000930740013306F60283A6460069
:103D70003307C7002322D7006FF0DFFB130101FEDA
:103D800023282101232E1100232C8100232A9100B6
:103D900023263101130905007370043097C4010014
:103DA0009384447183A7040017C401001304447270
:103DB000639C070C6314090003290400930949005C
:103DC00013850900EFC05FA183278902638607007E
:103DD00013058901EFC05FA09385090017D5010085
:103DE0001305858FEFC01F9783A704006388070022
:103DF0008327040083A747046394070A83270400EA
:103E00006384270D83A70400638207067370043060
:103E100083A704006398070E97C701009387076B79
:103E200003A70700032707006310070C9307F0FFA1
:103E300017C701002326F76683A7040063880702DB
:103E40008327040083A74704638207020327040033
:103E500083260400832747049387F7FF2322F70470
:103E600083A7460463940700736004308320C10174
:103E70000324810183244101032901018329C10015
:103E80001301010267800000032704008327040058
:103E900083274704938717002322F7046FF09FF1CD
:103EA0000327040083260400832747049387F7FF32
:103EB0002322F70483A74604E39207F473600430D7
:103EC00083270400E39027F583A704006382070695
:103ED00097C701009387875C83A707006388070A59
:103EE000737004306F00000083A7070083A7C7002A
:103EF00083A7C70083A7470017C701002322F75AEB
:103F00006FF09FF3032704008327040083274704EF
:103F1000938717002322F70497C701009387075B55
:103F200003A7070003270700E30207F06FF0DFFB9A
:103F300097C701009387C75817C701001307476841
:103F400083A70700032787116314F7028320C101A9
:103F50000324810197C7010023AC07568324410144
:103F6000032901018329C1001301010267800000B8
:103F7000032481018320C10183244101032901011C
:103F80008329C100130101026FF0DFCC03248101FA
:103F90008320C10183244101032901018329C10038
:103FA000130101026FC0CFDE6306050A130101FF92
:103FB0002322910097C4010093848451232021017E
:103FC0001389050083A50400232611002324810002
:103FD00093858501EFC00FFB03A504001305450081
:103FE000EFC08FFF9307F0FF630AF90697C7010040
:103FF0009387C74C03A4070003A7040083A7070007
:104000003304240123228700636EF40697C701005E
:104010009387C74B03A5070083A50400938545003C
:10402000EFC04FF697C701009387874783A7070024
:104030006376F40097C7010023A487468320C1005C
:10404000032481008324410003290100130101019D
:1040500067800000737004306F00000083A50400C7
:10406000032481008320C10083244100032901002F
:1040700017C501001305456693854500130101012D
:104080006FC04FED97C701009387074403A5070052
:104090000324810083A504008320C1008324410000
:1040A0000329010093854500130101016FC08FEDC5
:1040B000630E050097C701009387473E83A707005B
:1040C000639A0700737004306F000000737004304F
:1040D0006F000000130101FF2322910097C401002B
:1040E0009384043F03A704009387050083A504007D
:1040F000B7060080B3E7D7002326110023248100F0
:10410000232CF7009385850113040600EFC08FE48C
:1041100003A5040013054500EFC00FEC9307F0FF63
:104120006304F40297C701009387473903A507008A
:104130008320C100832441003305850003248100CE
:10414000130101016F40007D83A504000324810059
:104150008320C1008324410017C501001305C55702
:1041600093854500130101016FC0CFDE6308050A86
:10417000130101FF2322910097C401009384443569
:10418000232021011389050083A5040023261100A3
:10419000232481009385850113040600EFC08FDB83
:1041A00003A5040013054500EFC00FE393071000BB
:1041B000630AF40697C701009387473003A40700FA
:1041C00003A7040083A707003304240123228700E8
:1041D000636EF40697C701009387472F03A5070076
:1041E00083A5040093854500EFC0CFD997C7010090
:1041F0009387072B83A707006376F40097C7010016
:1042000023A0872A8320C100032481008324410046
:10421000032901001301010167800000737004305D
:104220006F00000083A50400032481008320C100E7
:10423000832441000329010017C501001305C54966
:1042400093854500130101016FC0CFD097C70100CE
:104250009387872703A507000324810083A5040013
:104260008320C10083244100032901009385450078
:10427000130101016FC00FD1130101FF23261100AB
:1042800023248100232291008327C50003A4C700B3
:104290006304040A9304840113850400EFC0CFD3A0
:1042A00097C701009387871F83A70700639A0708B2
:1042B0009304440013850400EFC00FD297C7010098
:1042C0009387871F0327C40283A7070063F6E700CD
:1042D00097C7010023A2E71E93172700B387E700C3
:1042E0009397270017C501001305852D93850400BA
:1042F0003305F500EFC00FC697C701009387471D30
:1043000083A707000327C4021305000083A7C70281
:1043100063FAE7009307100017C701002328F71876
:10432000130510008320C100032481008324410071
:104330001301010167800000737004306F000000FA
:104340009385040017C5010013058536EFC08FC0A3
:104350006FF09FFA97C701009387471483A7070060
:1043600063960700737004306F000000130101FFB3
:10437000232611002324810023229100B707008007
:104380000324C500B3E7F5002320F5006308040803
:10439000EFC08FC49304440013850400EFC0CFC363
:1043A00097C70100938747110327C40283A707001B
:1043B00063F6E70097C7010023A0E71093172700D3
:1043C000B387E7009397270017C501001305451F22
:1043D0003305F50093850400EFC0CFB797C7010000
:1043E0009387070F83A707000327C4021305000064
:1043F00083A7C70263FAE7009307100017C70100FD
:104400002326F70A130510008320C100032481002E
:1044100083244100130101016780000073700430A0
:104420006F0000006304050297C701009387C70768
:1044300003A7070097C701009387470883A70700D2
:104440002320E5002322F50067800000737004300C
:104450006F0000006304050E638E050C130101FF5D
:1044600023261100232481001307050073700430F4
:1044700097C801009388080483A708006380070297
:1044800097C701009387C70483A6070083A7070087
:1044900083A746049387170023A2F60417C30100DD
:1044A0001303C30183A70500032603009306F0FF4F
:1044B000130400006388D70417CE0100130ECEFE4C
:1044C00003250E0003280700832647006306A80083
:1044D000130410006378D6023308D640130410008A
:1044E0006372F80203250E00B387C740032603005A
:1044F000B387D70023A0F5002320A7002322C700FD
:104500001304000083A70800638C070097C701000D
:10451000938707FC83A7070083A7470463940702D8
:10452000130504008320C10003248100130101014D
:1045300067800000737004306F00000073700430F7
:104540006F000000EF4080456FF09FFD9307100063
:1045500017C70100232CF7F46780000063060500ED
:104560000325C50467800000130500006780000074
:10457000630405002326B5046780000097C7010087
:10458000938707F503A507006780000097C7010020
:10459000938747F283A7070013051000638C070079
:1045A00097C70100938787EF03A507001335150010
:1045B0001315150067800000630C0508130101FE48
:1045C000232A910097C40100938484F083A70400F8
:1045D000232E1100232C81002328210123263101C1
:1045E0000327C50283A7C7026376F70483278501E3
:1045F00063CC070083A7040083A6C7029307A0002B
:10460000B387D740232CF50093172700B387E70023
:104610000327450117C90100130989FA9397270059
:10462000B307F9006308F70283A7040083A7C70252
:104630002326F5028320C101032481018324410143
:10464000032901018329C1001301010267800000D1
:1046500067800000930945001304050013850900D5
:10466000EFC08F9783A7040017C701001307C7E4A3
:104670000327070083A7C7022326F4026376F70007
:1046800017C70100232AF7E2139527003305F50029
:1046900003248101131525008320C10183244101D6
:1046A000938509003305A9008329C100032901016D
:1046B000130101026FC00F8A63060502130101FF97
:1046C00023261100232481002322910097C7010093
:1046D000938707E003A40700630AA4007370043003
:1046E0006F00000013050000678000008327440569
:1046F00063960700737004306F0000008326C402C5
:10470000032704059387F7FF232AF4046384E60054
:10471000638E0700130500008320C100032481007D
:1047200083244100130101016780000093044400C9
:1047300013850400EFC04F8A8327040517C70100C3
:10474000130787D7832607001307A0003307F74016
:104750002326F402232CE40063F6F60017C70100B9
:10476000232CF7D413074001B387E70217C50100D4
:10477000130505E5938504003305F500EFB09FFDB3
:10478000130510006FF05FF97370043097C70100D4
:10479000938747D283A707006380070297C701006A
:1047A000938707D303A7070083A70700832747043E
:1047B000938717002322F7046780000097C7010042
:1047C000938747CF83A70700638C070297C7010031
:1047D000938707D003A70700032747046302070254
:1047E00003A7070083A60700832747049387F7FFE3
:1047F0002322F70483A74604639407007360043000
:104800006780000097C70100938787CC03A6070045
:1048100083A6070003A707009307A00083A6C6028C
:1048200003258601B387D740232CF700678000005B
:1048300097C701009387C7C903A70700630A07004A
:1048400083A6070003A746051307170023AAE6045B
:1048500003A5070067800000130101FD2320210349
:10486000232611022324810223229102232E3101C7
:10487000130905007370043097C40100938484C346
:1048800083A7040017C40100130484C4639E070AAD
:104890008327040083A78705639A07008327040002
:1048A0001307100023AEE704639A050E83A70400E4
:1048B000638807008327040083A74704639A0714CB
:1048C0007370043083A704006394070683270400F1
:1048D00003A5870563080500630209048327040014
:1048E00023AC07048327040023AE070483A7040036
:1048F000638807008327040083A7470463920706A1
:104900008320C1020324810283244102032901027E
:104910008329C101130101036780000003270400FC
:10492000832787059387F7FF232CF7046FF09FFBFE
:104930000327040083270400832747049387170075
:104940002322F7046FF09FF8032704008327040055
:1049500083274704938717002322F7046FF05FF340
:104960000327040083260400832747049387F7FF67
:104970002322F70483A74604E39407F87360043006
:104980008320C102032481028324410203290102FE
:104990008329C1011301010367800000032504007E
:1049A0002326B10013054500EFB01FE38325C100A6
:1049B0009307F0FF6380F50897C70100938707B05E
:1049C00083A907000327040083A70700B389B90060
:1049D0002322370163ECF90697C70100938707AFDD
:1049E00003A507008325040093854500EFB09FD9F8
:1049F00097C701009387C7AA83A7070063F6F9004A
:104A000097C7010023AE37A9EFB09FB86FF01FEA38
:104A10000327040083260400832747049387F7FFB6
:104A20002322F70483A74604E39C07E8736004305D
:104A30006FF01FE98325040017C501001305C5C9E0
:104A400093854500EFB01FD16FF01FFC97C70100A1
:104A5000938787A703A50700832504009385450056
:104A6000EFB05FD26FF05FFA130101FD2320210345
:104A7000232E3101232611022324810223229102B5
:104A8000232C41011389050093090600737004303B
:104A900097C40100938404A283A7040017C40100F3
:104AA000130404A3639C0714032704009307200046
:104AB0000327C7056304F702832704001345F5FFA6
:104AC00003A787053375E50023ACA70483270400FB
:104AD0001307100023AEE704639A060A83A70400B5
:104AE000638807008327040083A74704639407169D
:104AF0007370043083A70400639E0706638809006F
:104B00008327040083A7870523A0F9000327040057
:104B100093071000130500000327C705630EF70075
:104B2000832704001349F9FF1305100003A7870525
:104B30003379E90023AC27058327040023AE07045B
:104B400083A70400638807008327040083A7470422
:104B50006392070C8320C102032481028324410253
:104B6000032901028329C101032A810113010103E1
:104B7000678000000327040083270400832747047D
:104B8000938717002322F7046FF05FF703250400D3
:104B90002326D10013054500EFB01FC48326C100B2
:104BA0009307F0FF638AF60C97C70100938707917C
:104BB00003AA07000327040083A70700330ADA00CB
:104BC000232247016368FA0C97C701009387079077
:104BD00003A507008325040093854500EFB09FBA25
:104BE00097C701009387C78B83A707006370FA0AF2
:104BF00097C7010023A6478B6F00400903270400D5
:104C00008327040083274704938717002322F70490
:104C10006FF09FE9032704008326040083274704DD
:104C20009387F7FF2322F70483A74604E39407F250
:104C3000736004308320C102032481028324410273
:104C4000032901028329C101032A81011301010300
:104C5000678000000327040083260400832747049D
:104C60009387F7FF2322F70483A74604E39207E81C
:104C7000736004306FF0DFE78325040017C501007F
:104C8000130585A593854500EFB0DFACEFB05F90CD
:104C90006FF0DFE497C701009387078303A5070040
:104CA0008325040093854500EFB0DFAD6FF01FFE54
:104CB000630A050C130101FF232611002324810040
:104CC00023229100232021017370043097B4010046
:104CD0009384447E83A704006396070863860600D6
:104CE0008327850523A0F60093070600930620007E
:104CF0000326C505232ED5041387050013040500DC
:104D00006382D70A63F4F608930530006388B7001E
:104D1000930540006396B700630CD610232CE4047F
:104D200093071000630CF6081304100083A7040017
:104D3000638C070097B701009387877983A70700E3
:104D400083A7470463980706130504008320C10066
:104D50000324810083244100032901001301010180
:104D60006780000097B701009387877603A7070045
:104D700083A7070083274704938717002322F7049C
:104D80006FF0DFF5737004306F00000093061000C1
:104D9000E398D7F88327850533E7B700232CE5048C
:104DA0006FF01FF88327850593871700232CF504E0
:104DB0006FF01FF7EF30903E6FF01FF913094400BA
:104DC00013050900EFB05FA117B701001307C76E05
:104DD0008327C402032707006376F70017B7010093
:104DE000232CF76C13074001B387E70217B50100C6
:104DF0001305057D930509003305F500EFB09F9578
:104E00008327840263860700737004306F000000FC
:104E100097B701009387C76B83A707000327C402D6
:104E200083A7C702E3F2E7F0EFB08FF66FF0DFEF92
:104E3000130400006FF09FEF63080508130101FEE3
:104E4000232C8100232A91002328210123263101CC
:104E50002324410123225101232E1100930907002D
:104E6000138A060093040600138905001304050045
:104E7000EFB05F86930A050063060A008327840566
:104E80002320FA000327C40593072000232EF404EF
:104E90006380F40463FA9710930630006388D400AB
:104EA000930640006396D400630CF70E232C240570
:104EB000930710006312F70A8327840263820702B4
:104EC000737004306F000000737004306F000000D6
:104ED0008327840593871700232CF4046FF05FFD6C
:104EE00097B701009387875B83A707006390070A42
:104EF0009304440013850400EFB01F8E17B7010020
:104F00001307875B8327C402032707006376F70034
:104F100017B701002322F75A13074001B387E702AE
:104F200017B501001305C569938504003305F50025
:104F3000EFB05F8297B701009387875983A7070077
:104F40000327C40283A7C70263F8E700638609004A
:104F50009307100023A0F9001304100013850A0022
:104F6000EFB0CFF6130504008320C10103248101B3
:104F700083244101032901018329C100032A8100FF
:104F8000832A410013010102678000009305840118
:104F900017B501001305C571EFB0CFFB6FF09FF996
:104FA000130400006FF09FFB93071000E392F4F0EE
:104FB0008327840533E92701232C24056FF05FEF55
:104FC000630A050E130101FE232C8100232A9100A0
:104FD0001304050023282101232E1100232631016B
:104FE00093840500EFB00FEF930720008326C405DC
:104FF000232EF404832784051307100013090500EA
:1050000093871700232CF4046396E6088327840211
:1050100063860700737004306F00000097B70100CB
:105020009387C74783A70700639A0708930944003B
:1050300013850900EFB04FFA17B701001307C747F0
:105040008327C402032707006376F70017B7010020
:105050002324F74613074001B387E70217B5010081
:1050600013050556938509003305F500EFB08FEE63
:1050700097B701009387C74583A707000327C4029A
:1050800083A7C70263F8E700638604009307100054
:1050900023A0F400032481018320C1018324410162
:1050A0008329C1001305090003290101130101022D
:1050B0006FB0CFE1737004306F000000930584017E
:1050C00017B501001305C55EEFB0CFE86FF05FFACA
:1050D00093070500630805067370043017B70100D5
:1050E0001307473D83260700639E060203A6C705F4
:1050F00093062000130500006316D60023AE0704B4
:105100001305100083270700638C070097B7010081
:105110009387073C03A7070003274704631C070284
:105120006780000097B601009386863A03A60600C2
:1051300083A6060083264604938616002322D604FF
:105140006FF0DFFA97B701009387873883A70700CE
:105150006FF09FF803A7070083A607008327470483
:105160009387F7FF2322F70483A74604E39A07FAFD
:105170007360043067800000130101FB2322910457
:1051800023202105232C4103232A510323286103D3
:10519000232671032326110423248104232E3103A3
:1051A00023248103232291032320A10317B90100A3
:1051B0001309093317BB0100130BCB3197B401005E
:1051C0009384843197BA0100938A4A31130A1000FC
:1051D000930B90008327090003A7070063060716B7
:1051E00083A7C70083A90700EFD09FCFEFD0DFD000
:1051F00083270B00130C05006368F50C97B70100BB
:1052000023AAA72C130600006376352303A5040008
:10521000B3858941EFC01FCCEFE00F806306051610
:1052200003A5040093060000130600009305810007
:10523000EFC08FCAE30005FA83278100E3C207FEAF
:105240008329010183A7490163860700138549006B
:10525000EFB08FD8EFD05FCA83270B00130C050087
:105260006362F50C8327810017B701002324872789
:10527000E3E8FBFAB317FA0013F7072163100720DE
:1052800013F7770C6316072A93F70702E38A07F8E8
:1052900013850900EF00504F6FF09FF883A7C700F8
:1052A00003A4C70083AC07009309440013850900D9
:1052B000EFB08FD28327440213050400E780070074
:1052C0008327C4016386470D8327090003A70700CE
:1052D000E31607FC03A70A0097B6010023AC861F5C
:1052E00097B6010023ACF61E97B7010023AAE71E6C
:1052F000EFD09FF26FF0DFF283A7C70003A4C700CF
:1053000003AD0700930C440013850C00EFB0CFCC25
:105310008327440213050400E78007008327C401A4
:10532000638C470B8327090003A70700E31607FCDC
:1053300003A70A0097B6010023A2F61A97B7010047
:1053400023A0E71A6FF01FF2EFD09FB9EFD0DFBABA
:1053500083270B00130C0500E368F5F683A70A000A
:1053600003A504009309000003A60700B385894143
:1053700017B701002320871713361600EFC09FB51B
:10538000EFD09FE9E31E05E8EFB08FA06FF05FE973
:105390008327840193850900B387FC0063E2FC083E
:1053A00083A7040063860702232A0100232C9101AE
:1053B000232E8100EFF08F9D03A5040093060000CB
:1053C0001306000093054101EFB0CFF6E31E05EE92
:1053D000737004306F0000008327840193850C00F4
:1053E000B307FD006362FD0883A70400638607021C
:1053F000232A0100232CA101232E8100EFF00F9915
:1054000003A5040093060000130600009305410164
:10541000EFB04FF2E31805F0737004306F00000036
:10542000032509002322F40023288400EFB08FB560
:105430006FF09FE9EFD05FDE8327090083A7C700E5
:1054400003A4C700930C440013850C00EFB0CFB841
:105450008327C401638A4705832744021305040098
:10546000E78007006FF0DFDB032509002322F4004B
:1054700023288400EFB00FB16FF0DFEA8327C1006B
:1054800023ACF9006382070AB387870123A2F900DE
:1054900023A83901938549006362FC0803A50A002B
:1054A000EFB04FAE6FF0DFD783278401232884004D
:1054B0003387F9002322E400636AEC04330C3C4197
:1054C000636EFC0283A7040063860702232A01009F
:1054D000232C3101232E8100EFF04F8B03A5040014
:1054E000930600001306000093054101EFB08FE41E
:1054F000E31405F6737004306F00000003A50A0082
:1055000093850C00EFB00FA86FF01FF5032509007D
:1055100093850C00EFB00FA76FF01FF4032509006F
:10552000EFB04FA66FF0DFCF737004306F00000054
:105530008327C10083A6890123A839013387D700B7
:1055400023A2E9006362EC06B307FC4063EAD706D6
:1055500083A7490213850900E780070083A7C901D3
:10556000E39047CD83A689018327C10003A70400E8
:10557000B387D70063060702232A0100232CF1001A
:10558000232E3101EFF08F8003A504009306000065
:105590001306000093054101EFB0CFD9E31205C80F
:1055A000737004306F0000006374FC00E372F7FA5C
:1055B0000325090093854900EFB0CF9C6FF05FC6CB
:1055C00003A50A0093854900EFB0CF9B6FF05FC53C
:1055D000130101FF232481002326110023229100BF
:1055E0002320210117B40100130404EFEFF0CF9939
:1055F0008327040063840704EFF04F9C8327040093
:10560000638A070293080000130800009307000054
:1056100013072000930600001306004097B5010011
:105620009385C5D917050000130545B5EFC0DF9E6A
:1056300063140506737004306F00000017B9010091
:105640001309C90A13050900EFB04F8E97B4010082
:105650009384040B13850400EFB04F8D13060000F4
:105660009305C0001305400097B7010023AA27E760
:1056700097B7010023A497E6EFB0CFB717B70100A3
:10568000232CA7E46306050297B50100938585D214
:10569000EFC00FF16FF05FF68320C100032481009B
:1056A00083244100032901001301010167800000E8
:1056B000737004306F000000638A050A130101FD56
:1056C000232A5101930A05001305C00223248102F5
:1056D0002322910223202103232E3101232C410177
:1056E00023261102232861012326710113090700D3
:1056F00093890600130A060093840500EF00C0702A
:1057000013040500630C0502EFF00F8897B7010042
:10571000938787DC83A70700638E0704EFF00F8A67
:105720001305440023205401232C9400232E44010C
:105730002320340323222403EFB04F8113050400F8
:105740008320C10203248102832441020329010230
:105750008329C101032A8101832A4101032B01010D
:10576000832BC100130101036780000073700430B4
:105770006F00000097BB0100938B4BF713850B0064
:10578000EFA0DFFA17BB0100130B8BF713050B001B
:10579000EFA0DFF9130600009305C00013054000D9
:1057A00097B7010023AE77D397B7010023A867D33B
:1057B000EFB04FA417B701002320A7D2630A05005A
:1057C00097B50100938505BFEFC08FDD6FF01FF522
:1057D000737004306F000000630E0506130101FEB4
:1057E000232C8100232E1100232A910017B40100DD
:1057F000130484CE83280400130805001305000059
:1058000063800804930407002322B1001387060075
:105810002324C100232601019306500063C0B6046F
:10582000EFE0DFD693072000630EF50403250400A4
:10583000930600001306000093054100EFB08FAF00
:105840008320C1010324810183244101130101024A
:1058500067800000737004306F0000009305410002
:10586000930600001306070013850800EFB01FB968
:105870008320C1010324810183244101130101021A
:1058800067800000032504009306000013860400CF
:1058900093054100EFB00FAA6FF09FFA6306050071
:1058A0000325050067800000737004306F0000005E
:1058B00063160500737004306F000000130101FFD0
:1058C000232611002324810013040500EFE0DFEB01
:1058D000032544013334A000EFE05FEE130504001C
:1058E0008320C100032481001301010167800000AF
:1058F00063160500737004306F000000130101FF90
:10590000232481001304050023261100EFE0DFE7C4
:1059100003240402EFE09FEA8320C1001305040082
:105920000324810013010101678000006316050054
:10593000737004306F000000130101FF2324810005
:1059400023229100138405009304050023261100EF
:10595000EFE09FE323A08402032481008320C100A1
:1059600083244100130101016FE05FE5130101FF92
:105970001305C0012324810023261100EF00C04835
:1059800013040500630805002320050013054500E6
:10599000EFA0DFD9130504008320C1000324810098
:1059A000130101016780000063020502B70700FFD1
:1059B000B3F7F50063860700737004306F000000D2
:1059C000639A0500737004306F0000007370043038
:1059D0006F000000130101FE232C81002328210108
:1059E000232631012324410123225101232E1100BA
:1059F000232A91009309070013890600930A0600E1
:105A000013840500130A0500EFE05FB86318050072
:105A100063860900737004306F000000EFD04FCC34
:105A200083240A00B3779400631209046382070495
:105A300063880A009347F4FFB3F797002320FA0026
:105A4000EFD08FFD8320C101032481011385040061
:105A500003290101832441018329C100032A810014
:105A6000832A41001301010267800000E302F4FC75
:105A7000E38809FCB335500193958501630609005D
:105A8000B7070004B3E5F50013860900B3E5850008
:105A900013054A00EFE0CFE1EFD00FF863140500E3
:105AA000EFA01FAFEFE01FD6931765009309050025
:105AB00063DA0700B70400019384F4FFB3F499009C
:105AC0006FF05FF8EFE05FCC83290A00B377340111
:105AD00063100902638A070063880A009347F4FF92
:105AE000B3F737012320FA00EFE05FCD6FF09FFCA2
:105AF000E31CF4FE6FF05FFE630C0500B70700FFC8
:105B0000B3F7F500638A0700737004306F0000007C
:105B1000737004306F000000130101FF2324810023
:105B200013040500232611002322910023202101C4
:105B300013890500EFE05FC5832404009345F9FF56
:105B4000B3F795002320F400EFE05FC78320C10086
:105B500003248100138504000329010083244100EC
:105B60001301010167800000130101FF232481005C
:105B70001304050023261100EFA0DFB50324040061
:105B8000EFA0DFB48320C1001305040003248100CB
:105B90001301010167800000630C0500370700FF57
:105BA000B3F7E500638A0700737004306F000000EC
:105BB000737004306F0000006F201061B70700FFA2
:105BC000B377F60063860700737004306F0000003F
:105BD00063160600737004306F000000130101FEAD
:105BE000232C810023282101232631012324410174
:105BF000232E1100232A91001389060093890500A2
:105C0000130A050013040600EFE05F98631E050405
:105C100063060900737004306F000000EFD04FACD2
:105C200083240A009385090013050A00B3E4990050
:105C3000EFF09FF6B3779400630AF40883240A0018
:105C4000EFD08FDD8320C10103248101138504007F
:105C500003290101832441018329C100032A810012
:105C60001301010267800000EFD08FA783240A0090
:105C70009385090013050A00B3E43401EFF0DFF166
:105C8000B3F7840063848704E30A09FAB7050005C3
:105C900013060900B365B40013054A00EFE04FC1D5
:105CA000EFD08FD763140500EFA09F8EEFE09FB574
:105CB000931765009304050063D40702B70700013A
:105CC0009387F7FFB3F4F4006FF0DFF783270A0040
:105CD0001344F4FFB3F787002320FA006FF05FF658
:105CE000EFE09FAA83240A00B377940063988700AB
:105CF0009347F4FFB3F797002320FA00EFE01FACBF
:105D00006FF0DFFB130101FF232481002326110024
:105D10001304050023229100EFD08F9C83274400B9
:105D200063860702032504019304C40063189500E9
:105D30006F0080030325040163089502B705000284
:105D4000EFE04FE183274400E39607FE13050400CC
:105D5000EF008023032481008320C10083244100BD
:105D6000130101016FD04FCB737004306F0000003E
:105D7000630C0500370700FFB3F7E500638A0700EF
:105D8000737004306F000000737004306F00000007
:105D90006F209043630C0500B70700FFB3F7F500D1
:105DA000638A0700737004306F0000007370043062
:105DB0006F000000130101FF2324810023229100C2
:105DC000232611001304050093840500EFE0DF9BF8
:105DD0000327040093C7F4FFB377F7002320F400F0
:105DE000032481008320C1008324410013010101A9
:105DF0006FE0DF9C630605000325850167800000D6
:105E00001305000067800000130101FF23248100B7
:105E10002326110013040500EFD08F8C97A70100F3
:105E20009387476C83A70700639C0704B79701001B
:105E300017B701001307478E9387C7FF97A6010086
:105E400023A8E66A17A701002322F76A17B7010003
:105E50002326F78C97A701009387076917B70100DE
:105E6000232CF78A9307100017A701002324076843
:105E700017A70100232A076617A701002324F76646
:105E800063120402EFD04FB9EF10C05813040000A2
:105E9000130504008320C1000324810013010101C4
:105EA0006780000013058400937735006398070C22
:105EB000B79701001307F5FF9387A7FFE3E4E7FC1B
:105EC00097A601009386C66283A706006F00400173
:105ED00003A70700630A07009386070093070700DC
:105EE00003A74700E366A7FE17A701001307C75FD4
:105EF000E38AE7F803A7070013060001138487006D
:105F000023A0E60003A74700B306A740637ED6029E
:105F10003388A7002322D80023A2A70083254800A6
:105F200097A601009386C65C6F0080009306070069
:105F300003A7060003264700E36AB6FE2320E80015
:105F400023A0060103A7470097A701009387875D59
:105F500083A70700B387E74017A701002324F75C56
:105F6000EFD08FABE30204F2130504008320C100DD
:105F70000324810013010101678000001375C5FF30
:105F8000130545006FF0DFF263080506130101FFFA
:105F9000232481002326110013040500EFC05FF4C1
:105FA000930584FF0326C4FF17A701001307475476
:105FB0006F008000138707008327070083A6470030
:105FC000E3EAC6FE232CF4FE2320B70097A70100C6
:105FD0009387475503A707008327C4FF0324810045
:105FE0008320C100B387E70017A70100232CF752D5
:105FF000130101016FD04FA26780000097A7010035
:106000009387475203A50700678000006780000060
:106010003367B50013773700930705006312070451
:106020009308D6FFB30815011307050093860500F2
:106030006378150303A806001307470093864600FC
:10604000232E07FFE36817FF9347F5FFB387170178
:1060500093F7C7FF93874700B385F500B307F500B3
:106060003306C50063F4C70C9386450013884700C8
:10607000B3B6D70033B8050133E7F50093C6160071
:106080001348180013773700B3E6060113371700DB
:106090003377D700330EF640938617006308070660
:1060A0001337AE006314070613532E001388050040
:1060B00093860700130700008328080013071700C2
:1060C0001308480023A0160193864600E36667FE86
:1060D0001377CEFFB385E500B387E7006306EE04D0
:1060E00083C60500138717002380D700637EC7028D
:1060F00083C6150013872700A380D7006376C702E5
:1061000003C725002381E70067800000B307F6403E
:10611000B387F5009385150003C7F5FF9386160036
:10612000238FE6FEE398F5FE67800000678000009D
:10613000B367C50093F73700B308C5006382070E45
:1061400063761511B307A04093F737001387370024
:106150009306500093F5F50F130815003383A840FC
:106160001306F6FF6374D700130750006368E60E4A
:106170006380070E2300B50013071000638EE7004D
:10618000A300B50013073000130825006396E7004D
:10619000130835002301B5001396850033E6C500CA
:1061A000139705013367E6003303F34093968501A7
:1061B000B366D70013562300B307F500130700009A
:1061C00023A0D7001307170093874700E36AC7FE91
:1061D0001377C3FFB307E8006300E3082380B70029
:1061E00013871700637C1703A380B700138727006A
:1061F000637617032381B700138737006370170393
:10620000A381B70013874700637A17012382B70081
:106210001387570063741701A382B70067800000DB
:1062200093F5F50F13978500B365B7001397050134
:106230003367B700E37415FF9307050093874700A2
:1062400023AEE7FEE3EC17FF6780000067800000E5
:10625000130805006FF05FF46780000093070500E6
:106260006FF0DFF78347050013070500638C070015
:106270001305150083470500E39C07FE3305E54041
:1062800067800000130500006780000013051500FB
:106290008347F5FF9385150003C7F5FF6388070063
:1062A000E386E7FE3385E740678000009307000040
:1062B0006FF05FFF930705009385150003C7F5FF97
:1062C00093871700A38FE7FEE31807FE678000009F
:1062D00083460500930700026398F6001305150036
:1062E00083460500E38CF6FE938756FD93F7D70FA0
:1062F0006380070493070500930500006388060484
:106300001305000093871700138606FD1317250059
:1063100083C607003305A700131515003305A60033
:10632000E39206FE638405003305A0406780000009
:10633000938536FD8346150093B515009307150028
:10634000E39006FC130500006FF0DFFD130500006D
:106350006780000083A705002380A70083A70500AE
:106360009387170023A0F5006780000097A601001F
:106370009386861883A70600173703001307873C08
:1063800013861700B307F7002380A70097A5010025
:1063900023A4C5169307A000630AF5009307000421
:1063A0006308F6001305000067800000E30C06FE9A
:1063B000370610F0130717008347F7FF2320F6F086
:1063C00083A706009387F7FF97A5010023A6F51280
:1063D000E39207FE1305000067800000130101EB44
:1063E0002322911423202115232A511323248113BE
:1063F0002326111423248114232E3113232C41131B
:106400002328611323267113232291132320A11320
:10641000232EB11193040500138905002326C10022
:10642000130C5002930A9000834709006388870386
:10643000638C070603A404006F00800063860706D0
:106440002300F40003A4040013091900130414002A
:1064500023A0840083470900E39287FF03461900C5
:106460009308190093860800130D00029309F0FFAA
:10647000130AF0FF13080000130550059307D6FD1B
:1064800093F7F70F13891600636EF53A17A701000B
:10649000130747B793972700B387E70083A7070041
:1064A000B387E700678007008320C11403248114A9
:1064B00083244114032901148329C113032A81135E
:1064C000832A4113032B0113832BC112032C811246
:1064D000832C4112032D0112832DC11113010115CB
:1064E00067800000930C80002324010093071000B4
:1064F00063DA071D8327C10003A40400938B770090
:1065000093F68BFF03AB060083A9460093878600B2
:106510002326F10013860C009306000013050B00E0
:1065200093850900EF10107E2328A1009307000037
:1065300063803733930D4101930B100013860C00D9
:106540009306000013050B0093850900EF105038E7
:106550009306000013860C00130B050093890500B9
:10656000EF10507A8327810023A0AD0093861B0093
:10657000938D4D0063863701938B06006FF01FFCEF
:10658000E37C9BFF63D24603930704002380A701AB
:1065900003A40400130AFAFF9307140023A0F400D5
:1065A00013840700E3C446FF93962B009307010171
:1065B000B386D7006F008002938777052300F4002D
:1065C00003A40400938BFBFF93871B0013041400A8
:1065D00023A084009386C6FFE358F0E483A7060057
:1065E000E3ECFAFC938707036FF05FFD83A70400D9
:1065F000930600030327C1002380D70083A704006C
:1066000093064700930C00011386170023A0C400D3
:1066100013068007A380C70003A4040023240100FD
:10662000930707001304140023A0840003AB0700A2
:10663000930900002326D1006FF0DFED8327C1000E
:1066400083AC0700938B470063880C28635C40256C
:106650009307D002631EFD2083C70C0063880702E6
:1066600063D8092483A60400938C1C00130AFAFF44
:106670002380F60003A404001304140023A0840064
:1066800083C70C00E39E07FC6352400303A404008D
:10669000930700022300F40003A40400130AFAFF86
:1066A0001304140023A08400E3160AFE23267101BC
:1066B0006FF09FD72324010093071000930CA000D4
:1066C000E3CA07E38327C10003A4040093864700BD
:1066D0006FF0DFF503C61600930609006FF01FDAAE
:1066E00083A70400930650022380D70003A404006C
:1066F0001304140023A084006FF01FD3930C000137
:10670000232401006FF09FDE8327C10003C616001B
:106710009306090083A90700938747002326F10009
:10672000E35E0AD4138A09009309F0FF6FF01FD5C6
:1067300003C61600130DD002930609006FF01FD494
:106740009347FAFF93D7F74103C61600337AFA004E
:10675000930609006FF09FD203C61600130D0003C5
:10676000930609006FF09FD183C51600930906FDBB
:1067700093060900938705FD13860500E3E2FAFA04
:1067800093972900B38937019386160093991900CE
:10679000B389B90083C50600938909FD938705FD78
:1067A00013860500E3FEFAFC6FF09FF70327C10094
:1067B00083A7040083260700130747002326E10070
:1067C0002380D70003A404001304140023A0840032
:1067D0006FF09FC59307100063D4070F8327C10094
:1067E0009386770093F686FF938786002326F10031
:1067F00083A9460083A7060063DE090E83A6040072
:106800001306D002B307F0402380C60003A404009F
:10681000B336F000B30930411304140023A0840000
:10682000138B0700B389D940930CA00023240100E7
:106830006FF05FCE03C61600130818009306090018
:106840006FF0DFC383A70400138908006FF09FE98E
:10685000E3729BCF93071000930B00009306100088
:10686000E3C447D36FF05FD497AC0100938C8CB531
:106870009385090013850C00EF10C03D330AAA4030
:106880006352400303A404002300A40103A40400F2
:10689000130AFAFF1304140023A08400E3160AFE6F
:1068A000130A000083C70C00E38207E0E3CC09DA97
:1068B0009389F9FF1307F0FFE396E9DA6FF0DFDC65
:1068C0008327C1009386470083A707002326D100B2
:1068D00093D9F7416FF05FF2635640019307D002FE
:1068E000E314FDF897AC0100938CCCAD93078002C4
:1068F0006FF01FD7138B0700930CA0002324010017
:1069000003A404006FF01FC1130101EB232E311308
:10691000B70900409387F9FF23248114232291149F
:10692000232C4113232A511323261114232021152C
:106930002328611323267113232481132322911307
:106940002320A113232EB111130A05002324B10023
:1069500017A40100130444BA973A0300938A8ADE0D
:10696000979401009384847F2326F10093055002BD
:106970001305A00013080004B70610F083470A00AF
:10698000638EB7046388070A03270400130A1A00FA
:10699000130617003387EA0097A8010023AEC8B496
:1069A0002300F7006380A708E31A06FD17370300EA
:1069B000130747D9130717008347F7FF23A0F6F003
:1069C000832704009387F7FF17A601002326F6B25A
:1069D000E39207FE83470A00E396B7FA83461A005C
:1069E00013051A0013070500930B0002130BF0FFA9
:1069F000130CF0FF13080000930550059308900056
:106A00009387D6FD93F7F70F130A170063ECF5444D
:106A100093972700B387970083A70700B387970052
:106A200067800700173703001307C7D1E31406F880
:106A30006FF0DFF48320C1140324811483244114F4
:106A4000032901148329C113032A8113832A4113C3
:106A5000032B0113832BC112032C8112832C4112AF
:106A6000032D0112832DC111130101156780000050
:106A7000930C8000130D00009307100063DA0721C8
:106A8000832781009387770093F787FF83AD070003
:106A900003AB4700138787002324E10013860C0013
:106AA0009306000013850D0093050B00EF10902551
:106AB0002328A10063086D451309410193091000C3
:106AC00013860C009306000013850D0093050B0040
:106AD000EF10006013860C0093060000930D050074
:106AE000138B0500EF1010222320A90093891900B1
:106AF00013094900E3166DFDE3F49DFD1306000440
:106B0000B70610F063D489038327040013871700A6
:106B1000B387FA0097A5010023A0E59E23807701A3
:106B2000630AC706130CFCFFE3C089FF8327C1007B
:106B30001305C10093089000B386F90093962600D0
:106B400093070101B386D7001308A00013030004C4
:106B5000370610F0E38CA6E083A706009305000338
:106B600063F4F8009305700503270400B387B700AA
:106B7000930517003387EA0017AE0100232EBE9657
:106B80002300F70063860737638C65329386C6FF60
:106B90006FF05FFC173703001307C7BA130717001E
:106BA0008347F7FF23A0F6F0832704009387F7FFBE
:106BB00097A5010023A2F594E39207FE130CFCFFB6
:106BC0006FF09FF683270400130600041387170055
:106BD00097A5010023A2E592B386FA00930500036E
:106BE0002380B6006308C7509387270097A601004B
:106BF00023A4F6903387EA00930680072300D7008A
:106C000017370300130707B4B70610F06392C702E3
:106C1000130717008347F7FF23A0F6F0832704002C
:106C20009387F7FF17A601002328F68CE39207FE4F
:106C300083278100930C0001130D00009387470008
:106C400003278100130B0000832D07002324F1008C
:106C50006FF0DFE48327810083AC070013894700CE
:106C6000638E0C4C6358802B9307D0026394FB3ED9
:106C700003C70C00930507006314072A6F00002F59
:106C800093071000930CA000130D0000E3CA07DF68
:106C900083278100938747006FF09FFA8327810045
:106CA0008346170013070A0003AB070093874700CA
:106CB0002324F100E3560CD4130C0B00130BF0FF4C
:106CC0006FF01FD483461700930BD00213070A00FE
:106CD0006FF01FD39347FCFF93D7F741834617000C
:106CE000337CFC0013070A006FF09FD18346170026
:106CF000930B000313070A006FF09FD003461700A1
:106D0000138B06FD13070A00930706FD9306060082
:106D1000E3E2F8FA93172B00B38767011307170014
:106D200093971700B387C70003460700138B07FD2F
:106D3000930706FD93060600E3FEF8FC6FF09FF74D
:106D400083258100832704001306A00003A7050004
:106D500093861700B387FA0017950100232ED57884
:106D60002380E700138945006300C73693070004BA
:106D70006384F62A232421016FF05FBF930710007C
:106D800063DE07358327810013877700137787FF3A
:106D9000930787002324F100032B47008327070074
:106DA00063560B3E032704001306000493061700E6
:106DB0009795010023A2D5743387EA009305D0028A
:106DC0002300B700638CC638B307F0403337F000B8
:106DD000330B6041938D0700330BEB40930CA00005
:106DE000130D00006FF09FCB8346170013081800A7
:106DF00013070A006FF0DFC08346170013070A006D
:106E00006FF01FC083270400930600041387170048
:106E1000179601002322E66EB387FA00130650028C
:106E20002380C700E314D7B41737030013078791F3
:106E3000B70610F0130717008347F7FF23A0F6F0FB
:106E4000832704009387F7FF179601002326F66A2D
:106E5000E39207FE6FF09FB1930C0001130D000049
:106E60006FF09FC18327040093060004130A0500F6
:106E700013871700179601002320E668B387FA00EE
:106E8000130650022380C700E312D7AE1737030062
:106E90001307478BB70610F0130717008347F7FF58
:106EA00023A0F6F0832704009387F7FF17960100CD
:106EB0002324F664E39207FE130A05006FF01FAB6C
:106EC0001737030013070788130717008347F7FFD7
:106ED0002320F6F0832704009387F7FF979501009E
:106EE00023ACF560E39207FE9386C6FF6FF09FC662
:106EF0001737030013070785E39805FC9386C6FF41
:106F00006FF05FC5E3FA9DBB930910006FF01FBFE0
:106F1000130C000003C70C0093050700E30C07E403
:106F20009308F0FF1305A00013080004B70610F043
:106F3000635E0B0C8327040013861700B387FA00E7
:106F400017930100232AC35A2380E7006382A50810
:106F50006308060B938C1C0003C70C00130CFCFF8A
:106F600093050700E31607FCE35680E1832704003E
:106F70009305000213060004B70610F06F00C0006E
:106F8000130CFCFFE3080CDE13871700B387FA002D
:106F90002380B700179501002320E55693070700CB
:106FA000E310C7FE172703001307C779130717005D
:106FB0008347F7FF23A0F6F0832704009387F7FFAA
:106FC00017950100232AF552E39207FE6FF05FFB4D
:106FD0001727030013070777E30E06F613071700BA
:106FE0008347F7FF23A0F6F0832704009387F7FF7A
:106FF000179601002322F650E39207FE6FF09FF5EB
:1070000017270300130707746FF05FFD130BFBFFD7
:10701000E3121BF36FF05FF5172703001307877266
:10702000B70610F0130717008347F7FF23A0F6F009
:10703000832704009387F7FF17960100232EF64A53
:10704000E39207FE232421016FF05F92979C0100D9
:10705000938C4C3793050B0013850C00EF00903F89
:10706000330CAC40E35880EB832704001306000484
:10707000B70610F06F00C000130CFCFFE30A0CE829
:1070800013871700B387FA002380770197950100D3
:1070900023A4E54693070700E310C7FE1727030064
:1070A0001307476A130717008347F7FF23A0F6F07B
:1070B000832704009387F7FF9795010023AEF542DD
:1070C000E39207FE6FF05FFB172703001307876744
:1070D000E39806F4232421016FF05F898327810060
:1070E0001387470083A707002324E10013DBF74140
:1070F0006FF01FCB172703001307C764B70610F004
:10710000130717008347F7FF23A0F6F08327040037
:107110009387F7FF179601002320F63EE39207FEC0
:1071200093071000179701002328F73C9307800767
:10713000172703002308F7606FF09FAF63568001A5
:107140009307D002E394FBF0979C0100938C8C276B
:1071500013078002930580026FF09FDC97260300DF
:107160009386465E370610F09386160003C7F6FF37
:107170002320E6F0032704001307F7FF979501008B
:1071800023ACE536E31207FE6FF01FC4938D0700B2
:10719000930CA000130D00006FF05F90B70710F084
:1071A00023A0A7F26F000000130101FC13034102AA
:1071B0002322B10293050300232E11002324C102D0
:1071C0002326D1022328E102232AF102232C0103E2
:1071D000232E110323266100EFF00FF38320C1015A
:1071E000130500001301010467800000130101FB77
:1071F00013038103232481022326A100232CC1022F
:1072000013040500130603001305C1002326110211
:107210002322F104232ED1022320E104232401059B
:1072200023261105232E6100EFF04F9B8327C10019
:10723000238007000325C1008320C1023305854058
:10724000032481021301010567800000B70710F0D5
:1072500083A647F403A607F403A747F4E31AD7FE6F
:10726000B7260000938606F4B306D60033B6C600F0
:10727000B305E60023A4D7F423A6B7F46780000083
:10728000B70710F003A747F403A607F483A647F453
:10729000E31AD7FEB7260000938606F4B306D6009D
:1072A00033B6C60023A4D7F4B305E60023A6B7F48B
:1072B0009307000873A0473067800000130101FFA7
:1072C00023248100232611009797010093874723E9
:1072D000179401001304842203A7070083270400E6
:1072E0001306F07C9306470693874706979501009F
:1072F00023A8D5209795010023A2F520634AD60044
:107300008320C10003248100130101016780000074
:10731000130747899797010023A4E71EEF00D009C0
:10732000930710006316F50203270400B717000047
:107330009387F77613050000E3D4E7FCEFF01FE630
:10734000032481008320C100130101016FB05FB8E5
:107350001795010013058507EFF01FE513052000C1
:10736000EFF0DFE3032481008320C100130101015A
:107370006FB01FB617950100130505076FF0DFE228
:10738000179501001305C5066FF01FE2130101FFF9
:10739000232481002322910023261100B71400002A
:1073A00017940100130444059387843813000000E8
:1073B0009387F7FFE39C07FE13050400EFF0DFDE81
:1073C0006FF09FFE130500006F00C06D130101FFF9
:1073D00023261100EF00407E1307100093070000E2
:1073E000631AE5008320C100138507001301010122
:1073F0006780000017950100130545FDEFF0DFDA07
:107400008320C100930720001385070013010101A9
:1074100067800000737004306F0000006780000018
:10742000737004306F000000130101FF23248100FA
:1074300023261100179401001304C40D1305000046
:10744000EFC0DF938327040093871700179701008D
:107450002322F70C6FF09FFE130101FF232481000C
:107460002322910023261100930405001304100029
:1074700013050000EFC09F90930600001306F0FF75
:107480009305000013850400EF909FDB9306000036
:1074900013060000930500006302850213850400B3
:1074A0009797010023AE8706EF909FBAE30285FC11
:1074B0009797010023A687066FF09FFB93060000B5
:1074C000130600009305000013850400EF905FB8D9
:1074D000E30085FA9797010023A487046FF05FF912
:1074E000130101FE232C8100232A9100232821016E
:1074F000232631012324410123225101232061014C
:10750000232E110093090500179B0100130B4B005C
:10751000979A0100938A8AFF17990100130989FF3E
:10752000179A0100130A4AFF130410009304300055
:107530009306000013060000930500001385090060
:10754000EF901FD0630685009797010023AA87FC60
:10755000130500009797010023AE07FAEFB08F9B49
:10756000630605009797010023AC87FA03250B00FB
:10757000EFB08FC113050000EFB0CF9963069500FF
:107580009797010023AE87F81305000093051000BC
:10759000EFB04FA513050000EFB0CF97630695003D
:1075A0009797010023AE87F603A50A00EFB0CFBD81
:1075B00083270900638607009797010023A287F6B7
:1075C00093060000130600009305000013850900D0
:1075D000EF901FA8630685009797010023A287F408
:1075E00083270900638687009797010023AA87F203
:1075F00013050000EFB00F92630685009797010016
:1076000023A087F29305000013050000EFB08F9DC3
:1076100083270A009387170017970100232EF7EEA0
:107620006FF01FF1130101FC23244103179A01009D
:10763000130ACAEE232C8102232A91022328210354
:10764000232631032322510323206103232E7101BA
:10765000232E1102232C810113040500930B0A0031
:10766000130B200093044000930A50001309B0004C
:1076700093096000930610001306000093850B0029
:1076800013050400EF90DF9C13050400EFA0CFD892
:10769000930710006306F500179701002322F7E80F
:1076A00093060000130600009305810013050400F3
:1076B000EF901FB9930710006306F50017970100BC
:1076C0002320F7E603270A00832781006308F700D9
:1076D00093071000179701002324F7E41305040013
:1076E000EFA08FD3630805009307100017970100E0
:1076F0002328F7E2930600001306000093850B0091
:1077000013050400EF90DF9413050400EFA0CFD021
:10771000930710006306F500179701002322F7E096
:107720009306000013060000930581001305040072
:10773000EF901FB1930710006306F5001797010043
:107740002320F7DE13050400EFA00FCD630805002A
:1077500093071000179701002324F7DC03270A0082
:10776000832781006308F700930710001797010033
:107770002328F7DA23246101930600001306000092
:107780009305810013050400EF909F8C83278100EF
:10779000938717002324F100E3F0F4FE130504009F
:1077A000EFA08FC7930730006308F5009307100020
:1077B000179701002326F7D6930610001306000042
:1077C00093058100130C100013050400232481018C
:1077D000EF901F88930610001306000093058100A8
:1077E0001305040023240100EF909F861305040075
:1077F000EFA08FC2630655019797010023A287D39C
:107800009306100013060000930581001305040081
:10781000EF901F846308050093071000179701007D
:107820002320F7D093060000130600009305810083
:1078300013050400EF90DF81630805009307100033
:1078400017970100232EF7CC232401009306100084
:10785000130600009305C10013050400EF905F9E1E
:107860009307100093060000130600009305C10063
:107870006306F500179701002324F7CA8327C10088
:10788000032881001305040013C7F7FF6308F800FD
:1078900093071000179801002324F8C82326E1005D
:1078A000EF901F9A930710006306F50017970100E9
:1078B0002328F7C6832781008326C100138717007A
:1078C000638AD71C930710009796010023AAF6C479
:1078D0002324E100E3FCE4F613050400EFA0CFB39A
:1078E000630805009307100017970100232AF7C2C9
:1078F0009307A00093060000130600009305810083
:10790000130504002324F100EF908FF49307100077
:107910006306F500179701002324F7C093060000C3
:1079200013060000930581001305040023242101A0
:10793000EF900FF2930710006306F5001797010010
:107940002320F7BE13050400EFA00FAD6308650107
:1079500093071000179701002324F7BC93079000AA
:107960002324F10093061000130600009305810004
:1079700013050400EF90CFED930710006302F5109C
:1079800017970100232EF7B8832781009387F7FF0D
:107990002324F100E3E8F9FC13050400EFA0CFA7CE
:1079A000630855019307100017970100232AF7B6C3
:1079B00093061000130600009305810013050400D0
:1079C000EF900FE963080500930710001797010077
:1079D0002328F7B4930600001306000093058100E6
:1079E00013050400EF90CFE663080500930710002D
:1079F000179701002326F7B2930770002324F100A4
:107A0000130C100093060000130600009305C1003C
:107A100013050400EF90DF8263068501979701004C
:107A200023A087B1832781008326C1001387170015
:107A30006380D7049797010023A487AF2324E10034
:107A4000E372E9FC13050400EFA00F9D6308050035
:107A500093071000179701002324F7AC83270A002F
:107A60009387170017970100232AF7AA6FF09FC08A
:107A7000938717002324F100E376F9F86FF09FFC59
:107A8000832781009387F7FF2324F100E3ECF9ECCF
:107A90006FF09FF0938717002324F100E3F8F4DAE6
:107AA0006FF09FE3130101FF2322910013060000F2
:107AB0009304050093054000130550002326110090
:107AC00023248100EF801FF397950100938505948F
:107AD00013040500EFA0CFAC138704009306040045
:107AE00093080000130800009307000013060040ED
:107AF000979501009385C592170500001305C5B23F
:107B0000EFA08FD113051000EF90CFC39795010020
:107B10009385859113040500EFA08FA893060400B8
:107B200093080000130800009307000013070000EB
:107B300013060040979501009385C58F1705000037
:107B40001305459AEFA04FCD9308000013080000DD
:107B5000979701009387879B1307200093060000E7
:107B600013060040979501009385458D1705000089
:107B70001305C58BEFA04FCA9306040003248100B0
:107B80008320C100832441009308000013080000F3
:107B9000979701009387C79713073000130600409B
:107BA000979501009385058A170500001305058B3D
:107BB000130101016FA04FC6179701001307079625
:107BC00097960100938646948327070083A60600B4
:107BD0006398F600930710009796010023A2F6948D
:107BE0009797010093874793179601001306869194
:107BF00083A60700032606006308D60297960100B5
:107C0000938606920327070003A5060083A70700B3
:107C10009796010023AAE68E1335150017970100E9
:107C20002322F78E678000000327070083A7070041
:107C300093061000179601002324D68E130500002A
:107C40009796010023A2E68C17970100232CF78A50
:107C500067800000B305B500930705006386B70091
:107C600003C70700631607003385A740678000003D
:107C7000938717006FF09FFE9308000063DC0500F8
:107C80003305A040B337A000B305B040B385F5403D
:107C90009308F0FF63DA06003306C040B337C00034
:107CA000B306D040B386F6401308060013830600DF
:107CB0009307050013870500639806249786010043
:107CC0009386465F63F8C50E370E0100637AC60DD2
:107CD000130EF00F6374CE0013038000335E660052
:107CE000B386C60103CE0600330E6E0013030002F6
:107CF0003303C341630C0300B3956500335EC501D4
:107D0000331866003367BE00B3176500135E0801C1
:107D1000B355C703131508011355050193D6070181
:107D20003376C703B305B50213160601B366D60052
:107D300063FAB600B386060163E6060163F4B60093
:107D4000B3860601B386B64033F7C603939707019F
:107D500093D70701B3D6C603B306D502131507019F
:107D6000B367F50063FAD700B387070163E607013D
:107D700063F4D700B3870701B387D74033D56700D3
:107D800093050000638C0800B307A0403337F00070
:107D9000B305B04013850700B385E5406780000058
:107DA000370E000113030001E36AC6F313038001D9
:107DB0006FF0DFF2631606001308100033586802F4
:107DC000370701006372E80A1307F00F63740701B5
:107DD0001303800033576800B386E60003C606002D
:107DE00033066600130300023303C340631803081D
:107DF000B385054193560801131508011355050174
:107E000013D6070133F7D502B3D5D50213170701EF
:107E10003367C700B305B502637AB70033070701BC
:107E2000636607016374B70033070701B305B74002
:107E300033F7D5029397070193D70701B3D5D5023E
:107E4000B305B50213150701B367F50063FAB70070
:107E5000B387070163E6070163F4B700B38707013F
:107E6000B387B7406FF09FF137070001130300019C
:107E7000E362E8F6130380016FF0DFF53318680062
:107E800033DEC500935E08013356C500B3176500A5
:107E90003355DE03B39565003366B60093150801CC
:107EA00093D50501935606013377DE033385A5028A
:107EB000131707013367D700637AA7003307070159
:107EC000636607016374A70033070701B306A74081
:107ED00033F7D6031316060113560601B3D6D6039D
:107EE00013170701B386D502B365C70063FAD5003F
:107EF000B385050163E6050163F4D500B38505018B
:107F0000B385D5406FF01FEFE3EED5E637080100EB
:107F100063FC0605930EF00F33B8DE00131838002B
:107F200033DE0601178301001303C3383303C30193
:107F3000834E0300130E0002B38E0E01330EDE419A
:107F4000631E0E0263E4B600636AC500B307C54052
:107F5000B385D5403335F5003387A5401385070039
:107F6000930507006FF01FE23703000113080001BB
:107F7000E3E866FA130880016FF09FFA3357D601E1
:107F8000B396C601B366D700B357D50133D7D50131
:107F9000B395C501B3E7B70093D506013373B702B4
:107FA000139F0601135F0F0113D807013316C60193
:107FB0003315C5013357B7021313030133680301A7
:107FC000B30FEF0213030700637EF8013308D800F4
:107FD0001303F7FF6368D8006376F8011303E7FF24
:107FE0003308D8003308F841B37FB8023358B802D9
:107FF000939F0F01B3050F03139F0701135F0F0139
:1080000033EFEF0113070800637EBF00330FDF007B
:108010001307F8FF6368DF006376BF001307E8FF0C
:10802000330FDF0013130301B70F01003363E300C5
:108030009387FFFF13580601330FBF40B375F3005A
:1080400013530301B377F6003387F502B307F30246
:10805000B385050333030303B385F5001358070104
:108060003308B8006374F8003303F301B707010065
:108070009387F7FF935508013378F8001318080128
:108080003377F700B38565003307E8006366BF0008
:10809000631EBF00637CE5003306C7403337C7006B
:1080A000B385D540B385E540130706003307E540A7
:1080B0003335E500B305BF40B385A540B397D5017F
:1080C0003357C70133E5E700B3D5C5016FF09FCB48
:1080D00093870500130806001387060013030500A5
:1080E00063960628978801009388C81C63F6C50E1E
:1080F000370701006378E60C1307F00F3337C7002A
:1081000013173700B356E600B388D80083C60800BB
:108110003387E60093060002B386E640638C0600D0
:10812000B397D7003357E5003318D600B365F7008F
:108130003313D50013550801B3D7A5021316080150
:10814000135606019356030133F7A502B305F60251
:1081500013170701B366D7001387070063FEB60045
:10816000B38606011387F7FF63E8060163F6B600DE
:108170001387E7FFB3860601B386B640B3F7A602BE
:108180001313030113530301B3D6A60293970701F8
:1081900033E36700B305D60213850600637CB300A2
:1081A000330368001385F6FF636603016374B3004D
:1081B0001385E6FF131707013367A7009305000037
:1081C0006F00400EB706000113070001E36CD6F202
:1081D000130780016FF01FF363160600930610006B
:1081E00033D8C602B70601006372D80C9306F00FAD
:1081F00063F4060113078000B356E800B388D80083
:1082000083C60800B386E600130700023307D74091
:108210006318070AB3870741930510001356080136
:108220009318080193D808019356030133F7C70246
:10823000B3D7C70213170701B366D7003385F80217
:108240001387070063FEA600B38606011387F7FFB6
:1082500063E8060163F6A6001387E7FFB38606010D
:10826000B386A640B3F7C6021313030113530301E9
:10827000B3D6C6029397070133E36700B388D802E9
:1082800013850600637C1301330368001385F6FF32
:1082900063660301637413011385E6FF1317070177
:1082A0003367A7001305070067800000B7060001C9
:1082B00013070001E362D8F4130780016FF0DFF3C6
:1082C0003318E800B3D5D7003313E500B356D50013
:1082D00013550801B397E70033F7A502B3E8F6009A
:1082E0009317080193D7070113D60801B3D5A50248
:1082F000131707013367C700B386B702138605005B
:10830000637ED700330707011386F5FF6368070113
:108310006376D7001386E5FF33070701B306D7401E
:1083200033F7A6029398080193D80801B3D6A602A2
:1083300013170701B385D702B36717011387060028
:1083400063FEB700B38707011387F6FF63E80701F1
:1083500063F6B7001387E6FFB3870701B387B7401B
:1083600093150601B3E5E5006FF05FEB63E6D51802
:108370003707010063F4E6041308F00F3337D80021
:108380001317370033D8E60097850100938585F2EF
:10839000B385050103C80500930500023308E80012
:1083A000B38505416396050213071000E3ECF6EE72
:1083B0003335C500134715006FF0DFEEB705000138
:1083C00013070001E3E0B6FC130780016FF09FFB89
:1083D00033570601B396B600B366D70093DE0601A5
:1083E00033D70701B378D703B397B70033580501E4
:1083F0003363F8009397060193D7070113580301DD
:108400003316B6003357D7039398080133E80801B1
:10841000338FE702130E0700637EE8013308D800AC
:10842000130EF7FF6368D8006376E801130EE7FFC9
:108430003308D8003308E841B378D8033358D80359
:1084400093980801B38E07039317030193D707018D
:10845000B3E7F8001307080063FED701B387D7001E
:108460001307F8FF63E8D70063F6D7011307E8FFA7
:10847000B387D700131E0E01B387D741B70E010093
:108480003367EE001388FEFF33730701935807012B
:108490003378060113560601330E030333880803AD
:1084A00093560E013303C30233030301B386660000
:1084B000B388C80263F40601B388D80113D6060155
:1084C000B308160163E61703E39A17CFB707010055
:1084D0009387F7FFB3F6F60093960601337EFE000E
:1084E0003315B500B386C60193050000E37CD5DAE9
:1084F0001307F7FF6FF09FCC9305000013070000F0
:108500006FF05FDA930806001387060093070500F3
:1085100013880500639C062297860100938686D9FE
:1085200063FCC50C37030100637E660A1303F00F7A
:108530006374C300130780003353E600B3866600FC
:1085400003CE060013030002330EEE003303C341D3
:10855000630C0300B3956500335EC501B318660074
:108560003368BE00B317650013D608013377C8021D
:10857000139508011355050193D607013358C80216
:1085800013170701B366D7003308050363FA060122
:10859000B386160163E6160163F40601B38616017D
:1085A000B386064133F7C6029397070193D70701B5
:1085B000B3D6C602B306D50213150701B367F5009B
:1085C00063FAD700B387170163E6170163F4D70096
:1085D000B3871701B387D74033D5670093050000F1
:1085E000678000003703000113070001E36666F4AB
:1085F000130780016FF05FF4631606001306100086
:10860000B35816033706010063F2C80A1306F00FC9
:10861000637416011307800033D6E800B386C600E2
:1086200003CE060013030002330EEE003303C341F2
:1086300063180308B385154113D708011395080182
:108640001355050113D60701B3F6E502B3D5E502CC
:1086500093960601B3E6C600B305B50263FAB60009
:10866000B386160163E6160163F4B600B3861601FD
:10867000B385B640B3F6E5029397070193D7070198
:10868000B3D5E502B305B50213950601B367F5004E
:1086900063FAB700B387170163E6170163F4B70005
:1086A000B3871701B387B7406FF01FF33706000198
:1086B00013070001E3E2C8F6130780016FF0DFF54E
:1086C000B398680033D7C501B3176500335EC501A1
:1086D00013D50801B376A702B3956500336EBE00CB
:1086E0009395080193D5050113560E013357A70240
:1086F00093960601B3E6C6003387E50263FAE60007
:10870000B386160163E6160163F4E600B38616012C
:108710003386E640B376A602131E0E01135E0E01E9
:108720003356A602939606013386C502B3E5C60109
:1087300063FAC500B385150163E6150163F4C5004E
:10874000B3851501B385C5406FF01FEFE3EAD5E8A7
:108750003707010063FCE604930EF00F33B7DE0029
:108760001317370033D3E60097880100938888B445
:10877000B388680083CE0800130E0002B38EEE00AB
:10878000330EDE41631E0E0263E4B600636AC50069
:10879000B307C540B385D5403335F5003388A540D0
:1087A00013850700930508006FF09FE3B7080001E9
:1087B00013070001E3E816FB130780016FF09FFA2F
:1087C0003357D601B396C601B366D700B357D50168
:1087D00033D7D501B395C501B3E7B70093D50601EB
:1087E0003373B702139F0601135F0F0193D807017C
:1087F0003316C6013315C5013357B70213130301EE
:10880000B36813013308EF021303070063FE080186
:10881000B388D8001303F7FF63E8D80063F60801B4
:108820001303E7FFB388D800B3880841B3FFB80249
:10883000B3D8B802939F0F01B3051F03139F07011D
:10884000135F0F0133EFEF0113870800637EBF0052
:10885000330FDF001387F8FF6368DF006376BF0024
:108860001387E8FF330FDF0013130301B70801007C
:108870003363E3009387F8FF13580601330FBF40BB
:10888000B375F30013530301B377F6003387F50292
:10889000B307F302B385050333030303B385F50080
:1088A000135807013308B8006374F8003303130149
:1088B000B70701009387F7FF935508013378F80055
:1088C000131808013377F700B38565003307E80014
:1088D0006366BF00631EBF00637CE5003306C740CC
:1088E0003337C700B385D540B385E540130706008D
:1088F0003307E5403335E500B305BF40B385A540F8
:10890000B397D5013357C70133E5E700B3D5C501A8
:108910006FF01FCD97870100938787BB83A6070061
:1089200017870100130787B90327070023A2A600B2
:10893000637EE50017870100130707B903250700C9
:1089400083A50700938545006F70DFE3130101FFE6
:10895000232481002326110017870100130707B77E
:10896000130405000325070083A507009385450030
:10897000EF705FE197870100938787B283A70700B5
:108980006376F4009787010023AC87B08320C10091
:108990000324810013010101678000009787010013
:1089A000938707B303A7070083A60700832747041D
:1089B0009387F7FF2322F70483A7460463940700F5
:1089C0007360043067800000130101FE232C8100D6
:1089D000232A910013040500938405002328210114
:1089E000232631012324410123225101232E11008A
:1089F000EFA00FCF8327040003290401B70900016A
:108A0000B3E59700930AC4002320B4009304000048
:108A10009389F9FF370A00020327040063822A05BD
:108A20000326090013050900B3654701B376360133
:108A30009317560033F7E6000329490063C6070081
:108A4000631607006FF05FFDE398E6FC931776006E
:108A500063D40700B3E4D400EFB0DF8F6FF0DFFB27
:108A600093C4F4FFB3F4E40023209400EFA0CFFA02
:108A7000032504008320C1010324810183244101D3
:108A8000032901018329C100032A8100832A4100AF
:108A90001301010267800000130101FF13050000AC
:108AA0002326110023248100EFE0DFFF17F7FFFFEB
:108AB0001307078193060000130610009305200397
:108AC000178501001305C593EFC01FBF63020502A0
:108AD00013040500EFA04FC21306050013070000A2
:108AE000930600009305100013050400EFC0DFCECD
:108AF000EFA04F8C8320C1000324810013050000E8
:088B0000130101016780000070
:02000004800278
:10000000D466FEFF4468FEFFE066FEFF4468FEFF24
:100010004468FEFF4468FEFF4468FEFF0867FEFF79
:100020004468FEFF4468FEFF3067FEFF4067FEFF46
:100030004468FEFF5867FEFF6867FEFF6867FEFFC3
:100040006867FEFF6867FEFF6867FEFF6867FEFF80
:100050006867FEFF6867FEFF6867FEFF4468FEFF93
:100060004468FEFF4468FEFF4468FEFF4468FEFFEC
:100070004468FEFF4468FEFF4468FEFF4468FEFFDC
:100080004468FEFF4468FEFF4468FEFF4468FEFFCC
:100090004468FEFF4468FEFF4468FEFF4468FEFFBC
:1000A0004468FEFF4468FEFF4468FEFF4468FEFFAC
:1000B0004468FEFF4468FEFF4468FEFF4468FEFF9C
:1000C0004468FEFF4468FEFF4468FEFF4468FEFF8C
:1000D0004468FEFF4468FEFF4468FEFF4468FEFF7C
:1000E0004468FEFF4468FEFF4468FEFF4468FEFF6C
:1000F0004468FEFF4468FEFF4468FEFF4468FEFF5C
:10010000AC67FEFFD467FEFF4468FEFF4468FEFF55
:100110004468FEFF4468FEFF4468FEFF4468FEFF3B
:100120004468FEFF3468FEFF4468FEFF4468FEFF3B
:10013000E464FEFFEC65FEFF4468FEFF4468FEFFDA
:100140003C66FEFF4468FEFFB466FEFF4468FEFFA7
:100150004468FEFFFC66FEFFA06CFEFF0C6DFEFF18
:10016000AC6CFEFF0C6DFEFF0C6DFEFF0C6DFEFF18
:100170000C6DFEFF446BFEFF0C6DFEFF0C6DFEFF71
:100180006C6BFEFF7C6BFEFF0C6DFEFF946BFEFF45
:10019000A46BFEFFA46BFEFFA46BFEFFA46BFEFF2F
:1001A000A46BFEFFA46BFEFFA46BFEFFA46BFEFF1F
:1001B000A46BFEFF0C6DFEFF0C6DFEFF0C6DFEFFD1
:1001C0000C6DFEFF0C6DFEFF0C6DFEFF0C6DFEFF57
:1001D0000C6DFEFF0C6DFEFF0C6DFEFF0C6DFEFF47
:1001E0000C6DFEFF0C6DFEFF0C6DFEFF0C6DFEFF37
:1001F0000C6DFEFF0C6DFEFF0C6DFEFF0C6DFEFF27
:100200000C6DFEFF0C6DFEFF0C6DFEFF0C6DFEFF16
:100210000C6DFEFF0C6DFEFF0C6DFEFF0C6DFEFF06
:100220000C6DFEFF0C6DFEFF0C6DFEFF0C6DFEFFF6
:100230000C6DFEFF0C6DFEFF0C6DFEFF0C6DFEFFE6
:100240000C6DFEFF0C6DFEFF0C6DFEFF0C6DFEFFD6
:100250000C6DFEFF0C6DFEFFE86BFEFF246CFEFFD5
:100260000C6DFEFF0C6DFEFF0C6DFEFF0C6DFEFFB6
:100270000C6DFEFF0C6DFEFF0C6DFEFF906CFEFF23
:100280000C6DFEFF0C6DFEFF1869FEFF6C6AFEFF31
:100290000C6DFEFF0C6DFEFFFC6AFEFF0C6DFEFF99
:1002A000286BFEFF0C6DFEFF0C6DFEFF006DFEFF68
:1002B000000102020303030304040404040404040D
:1002C00005050505050505050505050505050505DE
:1002D00006060606060606060606060606060606BE
:1002E00006060606060606060606060606060606AE
:1002F000070707070707070707070707070707078E
:10030000070707070707070707070707070707077D
:10031000070707070707070707070707070707076D
:10032000070707070707070707070707070707075D
:10033000080808080808080808080808080808083D
:10034000080808080808080808080808080808082D
:10035000080808080808080808080808080808081D
:10036000080808080808080808080808080808080D
:1003700008080808080808080808080808080808FD
:1003800008080808080808080808080808080808ED
:1003900008080808080808080808080808080808DD
:1003A00008080808080808080808080808080808CD
:1003B000546D725100000000546D7220537663003A
:1003C000286E756C6C2900004572726F7220696E20
:1003D00020416C745154657374207461736B732085
:1003E0000D0A00006D69616F750A00006D69616F2B
:1003F00075320A0068756E6772790A004368656332
:100400006B54696D65720000416C745F47656E5F87
:10041000546573745F517565756500004647656E78
:1004200051000000416C745F515F4D757465780038
:10043000464D754C6F770000464D754D6564000064
:08044000464D7548696768002C
:100448001000000000000000017A5200017C010148
:100458001B0D020010000000180000001478FEFFB9
:100468005804000000000000100000002C000000EC
:10047800587CFEFF3404000000000000100000005B
:10048800400000007880FEFF10040000000000001B
:08052000FC8F0100090000003E
:040000058000004037
:00000001FF
